 jsound

 Timestamp is 8a067875 (reproducible build file hash)

 Preferred load address is 0000000180000000

 Start         Length     Name                   Class
 0001:00000000 00000040H .text$di                CODE
 0001:00000040 00007ba0H .text$mn                CODE
 0001:00007be0 00000036H .text$mn$00             CODE
 0001:00007c16 00000092H .text$x                 CODE
 0001:00007ca8 00000018H .text$yd                CODE
 0002:00000000 00000330H .idata$5                DATA
 0002:00000330 00000038H .00cfg                  DATA
 0002:00000368 00000008H .CRT$XCA                DATA
 0002:00000370 00000010H .CRT$XCU                DATA
 0002:00000380 00000008H .CRT$XCZ                DATA
 0002:00000388 00000008H .CRT$XIA                DATA
 0002:00000390 00000008H .CRT$XIZ                DATA
 0002:00000398 00000008H .CRT$XPA                DATA
 0002:000003a0 00000008H .CRT$XPZ                DATA
 0002:000003a8 00000008H .CRT$XTA                DATA
 0002:000003b0 00000010H .CRT$XTZ                DATA
 0002:000003b8 00000000H .gehcont$y              DATA
 0002:000003b8 00000000H .gfids$y                DATA
 0002:000003c0 00000840H .rdata                  DATA
 0002:00000c00 00000000H .rdata$CastGuardVftablesA DATA
 0002:00000c00 00000000H .rdata$CastGuardVftablesC DATA
 0002:00000c00 000001f4H .rdata$r                DATA
 0002:00000df4 0000010cH .rdata$voltmd           DATA
 0002:00000f00 00000340H .rdata$zzzdbg           DATA
 0002:00001240 00000008H .rtc$IAA                DATA
 0002:00001248 00000008H .rtc$IZZ                DATA
 0002:00001250 00000008H .rtc$TAA                DATA
 0002:00001258 00000008H .rtc$TZZ                DATA
 0002:00001260 000005b0H .xdata                  DATA
 0002:00001810 000000f0H .xdata$x                DATA
 0002:00001900 00000cecH .edata                  DATA
 0002:000025ec 000000c8H .idata$2                DATA
 0002:000026b4 00000014H .idata$3                DATA
 0002:000026c8 00000330H .idata$4                DATA
 0002:000029f8 00000768H .idata$6                DATA
 0003:00000000 00000058H .data                   DATA
 0003:00000058 00000080H .data$r                 DATA
 0003:000000d8 00000028H .data$rs                DATA
 0003:00000100 000011c0H .bss                    DATA
 0004:00000000 00000924H .pdata                  DATA
 0005:00000000 00000060H .rsrc$01                DATA
 0005:00000060 00000328H .rsrc$02                DATA

  Address         Publics by Value              Rva+Base               Lib:Object

 0000:00000000       __AbsoluteZero             0000000000000000     <absolute>
 0000:00000000       ___safe_se_handler_count   0000000000000000     <absolute>
 0000:00000000       ___safe_se_handler_table   0000000000000000     <absolute>
 0000:00000000       __arm64x_extra_rfe_table   0000000000000000     <absolute>
 0000:00000000       __arm64x_extra_rfe_table_size 0000000000000000     <absolute>
 0000:00000000       __arm64x_native_entrypoint 0000000000000000     <absolute>
 0000:00000000       __arm64x_redirection_metadata 0000000000000000     <absolute>
 0000:00000000       __arm64x_redirection_metadata_count 0000000000000000     <absolute>
 0000:00000000       __dynamic_value_reloc_table 0000000000000000     <absolute>
 0000:00000000       __enclave_config           0000000000000000     <absolute>
 0000:00000000       __guard_check_icall_a64n_fptr 0000000000000000     <absolute>
 0000:00000000       __guard_eh_cont_count      0000000000000000     <absolute>
 0000:00000000       __guard_eh_cont_table      0000000000000000     <absolute>
 0000:00000000       __guard_fids_count         0000000000000000     <absolute>
 0000:00000000       __guard_fids_table         0000000000000000     <absolute>
 0000:00000000       __guard_iat_count          0000000000000000     <absolute>
 0000:00000000       __guard_iat_table          0000000000000000     <absolute>
 0000:00000000       __guard_longjmp_count      0000000000000000     <absolute>
 0000:00000000       __guard_longjmp_table      0000000000000000     <absolute>
 0000:00000000       __hybrid_auxiliary_delayload_iat 0000000000000000     <absolute>
 0000:00000000       __hybrid_auxiliary_delayload_iat_copy 0000000000000000     <absolute>
 0000:00000000       __hybrid_auxiliary_iat     0000000000000000     <absolute>
 0000:00000000       __hybrid_auxiliary_iat_copy 0000000000000000     <absolute>
 0000:00000000       __hybrid_code_map          0000000000000000     <absolute>
 0000:00000000       __hybrid_code_map_count    0000000000000000     <absolute>
 0000:00000000       __hybrid_image_info_bitfield 0000000000000000     <absolute>
 0000:00000000       __x64_code_ranges_to_entry_points 0000000000000000     <absolute>
 0000:00000000       __x64_code_ranges_to_entry_points_count 0000000000000000     <absolute>
 0000:00000100       __guard_flags              0000000000000100     <absolute>
 0000:00000000       __ImageBase                0000000180000000     <linker-defined>
 0001:00000040       DAUDIO_AddAudioFormat      0000000180001040 f   DirectAudioDevice.obj
 0001:000000d0       Java_com_sun_media_sound_DirectAudioDevice_nAvailable 00000001800010d0 f   DirectAudioDevice.obj
 0001:000000f4       Java_com_sun_media_sound_DirectAudioDevice_nClose 00000001800010f4 f   DirectAudioDevice.obj
 0001:00000130       Java_com_sun_media_sound_DirectAudioDevice_nFlush 0000000180001130 f   DirectAudioDevice.obj
 0001:00000150       Java_com_sun_media_sound_DirectAudioDevice_nGetBufferSize 0000000180001150 f   DirectAudioDevice.obj
 0001:00000174       Java_com_sun_media_sound_DirectAudioDevice_nGetBytePosition 0000000180001174 f   DirectAudioDevice.obj
 0001:0000019c       Java_com_sun_media_sound_DirectAudioDevice_nGetFormats 000000018000119c f   DirectAudioDevice.obj
 0001:00000200       Java_com_sun_media_sound_DirectAudioDevice_nIsStillDraining 0000000180001200 f   DirectAudioDevice.obj
 0001:0000022c       Java_com_sun_media_sound_DirectAudioDevice_nOpen 000000018000122c f   DirectAudioDevice.obj
 0001:00000344       Java_com_sun_media_sound_DirectAudioDevice_nRead 0000000180001344 f   DirectAudioDevice.obj
 0001:000003fc       Java_com_sun_media_sound_DirectAudioDevice_nRequiresServicing 00000001800013fc f   DirectAudioDevice.obj
 0001:00000420       Java_com_sun_media_sound_DirectAudioDevice_nService 0000000180001420 f   DirectAudioDevice.obj
 0001:00000440       Java_com_sun_media_sound_DirectAudioDevice_nSetBytePosition 0000000180001440 f   DirectAudioDevice.obj
 0001:00000464       Java_com_sun_media_sound_DirectAudioDevice_nStart 0000000180001464 f   DirectAudioDevice.obj
 0001:00000484       Java_com_sun_media_sound_DirectAudioDevice_nStop 0000000180001484 f   DirectAudioDevice.obj
 0001:000004a4       Java_com_sun_media_sound_DirectAudioDevice_nWrite 00000001800014a4 f   DirectAudioDevice.obj
 0001:000006d4       handleGainAndConversion    00000001800016d4 f   DirectAudioDevice.obj
 0001:00001c00       handleSignEndianConversion 0000000180002c00 f   DirectAudioDevice.obj
 0001:00001cf0       Java_com_sun_media_sound_DirectAudioDeviceProvider_nGetNumDevices 0000000180002cf0 f   DirectAudioDeviceProvider.obj
 0001:00001cf8       Java_com_sun_media_sound_DirectAudioDeviceProvider_nNewDirectAudioDeviceInfo 0000000180002cf8 f   DirectAudioDeviceProvider.obj
 0001:00001e60       getDirectAudioDeviceDescription 0000000180002e60 f   DirectAudioDeviceProvider.obj
 0001:00001edc       Java_com_sun_media_sound_MidiInDevice_nClose 0000000180002edc f   MidiInDevice.obj
 0001:00001ee4       Java_com_sun_media_sound_MidiInDevice_nGetMessages 0000000180002ee4 f   MidiInDevice.obj
 0001:00002114       Java_com_sun_media_sound_MidiInDevice_nGetTimeStamp 0000000180003114 f   MidiInDevice.obj
 0001:00002114       Java_com_sun_media_sound_MidiOutDevice_nGetTimeStamp 0000000180003114 f   MidiOutDevice.obj
 0001:00002130       Java_com_sun_media_sound_MidiInDevice_nOpen 0000000180003130 f   MidiInDevice.obj
 0001:00002184       Java_com_sun_media_sound_MidiInDevice_nStart 0000000180003184 f   MidiInDevice.obj
 0001:000021b8       Java_com_sun_media_sound_MidiInDevice_nStop 00000001800031b8 f   MidiInDevice.obj
 0001:000021c0       Java_com_sun_media_sound_MidiInDeviceProvider_nGetDescription 00000001800031c0 f   MidiInDeviceProvider.obj
 0001:0000223c       Java_com_sun_media_sound_MidiInDeviceProvider_nGetName 000000018000323c f   MidiInDeviceProvider.obj
 0001:000022b8       Java_com_sun_media_sound_MidiInDeviceProvider_nGetNumDevices 00000001800032b8 f   MidiInDeviceProvider.obj
 0001:000022c0       Java_com_sun_media_sound_MidiInDeviceProvider_nGetVendor 00000001800032c0 f   MidiInDeviceProvider.obj
 0001:000022c0       Java_com_sun_media_sound_MidiOutDeviceProvider_nGetVendor 00000001800032c0 f   MidiOutDeviceProvider.obj
 0001:0000233c       Java_com_sun_media_sound_MidiInDeviceProvider_nGetVersion 000000018000333c f   MidiInDeviceProvider.obj
 0001:000023b8       Java_com_sun_media_sound_MidiOutDevice_nClose 00000001800033b8 f   MidiOutDevice.obj
 0001:000023c0       Java_com_sun_media_sound_MidiOutDevice_nOpen 00000001800033c0 f   MidiOutDevice.obj
 0001:0000240c       Java_com_sun_media_sound_MidiOutDevice_nSendLongMessage 000000018000340c f   MidiOutDevice.obj
 0001:00002494       Java_com_sun_media_sound_MidiOutDevice_nSendShortMessage 0000000180003494 f   MidiOutDevice.obj
 0001:000024a4       Java_com_sun_media_sound_MidiOutDeviceProvider_nGetDescription 00000001800034a4 f   MidiOutDeviceProvider.obj
 0001:00002520       Java_com_sun_media_sound_MidiOutDeviceProvider_nGetName 0000000180003520 f   MidiOutDeviceProvider.obj
 0001:0000259c       Java_com_sun_media_sound_MidiOutDeviceProvider_nGetNumDevices 000000018000359c f   MidiOutDeviceProvider.obj
 0001:000025a4       Java_com_sun_media_sound_MidiOutDeviceProvider_nGetVersion 00000001800035a4 f   MidiOutDeviceProvider.obj
 0001:00002620       UnicodeToUTF8              0000000180003620 f   PLATFORM_API_WinOS_Charset_Util.obj
 0001:000026b8       UnicodeToUTF8AndCopy       00000001800036b8 f   PLATFORM_API_WinOS_Charset_Util.obj
 0001:00002708       ??0Data@DS_StartBufferHelper@@QEAA@XZ 0000000180003708 f   PLATFORM_API_WinOS_DirectSound.obj
 0001:00002788       ??1Data@DS_StartBufferHelper@@QEAA@XZ 0000000180003788 f   PLATFORM_API_WinOS_DirectSound.obj
 0001:000027d0       ?DS_CheckUnderrun@@YAXPEAUDS_Info@@KK@Z 00000001800037d0 f   PLATFORM_API_WinOS_DirectSound.obj
 0001:00002800       ?DS_GetAvailable@@YAHPEAUDS_Info@@PEAK1PEAHH@Z 0000000180003800 f   PLATFORM_API_WinOS_DirectSound.obj
 0001:00002958       ?DS_GetDescEnum@@YAHPEAU_GUID@@PEBG1PEAUtag_DirectAudioDeviceDescription@@@Z 0000000180003958 f   PLATFORM_API_WinOS_DirectSound.obj
 0001:000029ac       ?DS_RefreshCacheEnum@@YAHPEAU_GUID@@PEBD1PEAUDS_RefreshCacheStruct@@@Z 00000001800039ac f   PLATFORM_API_WinOS_DirectSound.obj
 0001:00002a50       ?DS_addDeviceRef@@YAHH@Z   0000000180003a50 f   PLATFORM_API_WinOS_DirectSound.obj
 0001:00002b28       ?DS_clearBuffer@@YAXPEAUDS_Info@@H@Z 0000000180003b28 f   PLATFORM_API_WinOS_DirectSound.obj
 0001:00002d1c       ?DS_createSoundBuffer@@YAPEAXPEAUDS_Info@@MHHH@Z 0000000180003d1c f   PLATFORM_API_WinOS_DirectSound.obj
 0001:00002e38       ?DS_destroySoundBuffer@@YAXPEAUDS_Info@@@Z 0000000180003e38 f   PLATFORM_API_WinOS_DirectSound.obj
 0001:00002e70       ?DS_removeDeviceRef@@YAXH@Z 0000000180003e70 f   PLATFORM_API_WinOS_DirectSound.obj
 0001:00002ec0       ?StartBuffer@DS_StartBufferHelper@@SAJPEAUDS_Info@@@Z 0000000180003ec0 f   PLATFORM_API_WinOS_DirectSound.obj
 0001:00002f28       ?ThreadProc@DS_StartBufferHelper@@KAKPEAX@Z 0000000180003f28 f   PLATFORM_API_WinOS_DirectSound.obj
 0001:00002fa8       ?createWaveFormat@@YAXPEAUWAVEFORMATEXTENSIBLE@@HHHH@Z 0000000180003fa8 f   PLATFORM_API_WinOS_DirectSound.obj
 0001:00003048       ?findCacheItemByGUID@@YAHPEAU_GUID@@H@Z 0000000180004048 f   PLATFORM_API_WinOS_DirectSound.obj
 0001:000030c4       ?findCacheItemByMixerIndex@@YAHH@Z 00000001800040c4 f   PLATFORM_API_WinOS_DirectSound.obj
 0001:000030ec       ?isEqualGUID@@YAHPEAU_GUID@@0@Z 00000001800040ec f   PLATFORM_API_WinOS_DirectSound.obj
 0001:00003138       DAUDIO_Close               0000000180004138 f   PLATFORM_API_WinOS_DirectSound.obj
 0001:00003160       DAUDIO_Flush               0000000180004160 f   PLATFORM_API_WinOS_DirectSound.obj
 0001:000031c0       DAUDIO_GetAvailable        00000001800041c0 f   PLATFORM_API_WinOS_DirectSound.obj
 0001:000031e4       DAUDIO_GetBufferSize       00000001800041e4 f   PLATFORM_API_WinOS_DirectSound.obj
 0001:000031e8       DAUDIO_GetBytePosition     00000001800041e8 f   PLATFORM_API_WinOS_DirectSound.obj
 0001:00003234       DAUDIO_GetDirectAudioDeviceCount 0000000180004234 f   PLATFORM_API_WinOS_DirectSound.obj
 0001:00003340       DAUDIO_GetDirectAudioDeviceDescription 0000000180004340 f   PLATFORM_API_WinOS_DirectSound.obj
 0001:000033cc       DAUDIO_GetFormats          00000001800043cc f   PLATFORM_API_WinOS_DirectSound.obj
 0001:000034c4       DAUDIO_Open                00000001800044c4 f   PLATFORM_API_WinOS_DirectSound.obj
 0001:00003618       DAUDIO_Read                0000000180004618 f   PLATFORM_API_WinOS_DirectSound.obj
 0001:00003744       DAUDIO_RequiresServicing   0000000180004744 f   PLATFORM_API_WinOS_DirectSound.obj
 0001:0000374c       DAUDIO_Service             000000018000474c f   PLATFORM_API_WinOS_DirectSound.obj
 0001:00003794       DAUDIO_SetBytePosition     0000000180004794 f   PLATFORM_API_WinOS_DirectSound.obj
 0001:00003794       _guard_check_icall_nop     0000000180004794 f   MSVCRT:guard_support.obj
 0001:00003798       DAUDIO_Start               0000000180004798 f   PLATFORM_API_WinOS_DirectSound.obj
 0001:00003848       DAUDIO_StillDraining       0000000180004848 f   PLATFORM_API_WinOS_DirectSound.obj
 0001:0000388c       DAUDIO_Stop                000000018000488c f   PLATFORM_API_WinOS_DirectSound.obj
 0001:000038c0       DAUDIO_Write               00000001800048c0 f   PLATFORM_API_WinOS_DirectSound.obj
 0001:00003a78       ??0Data@MidiIn_OpenHelper@@QEAA@XZ 0000000180004a78 f   PLATFORM_API_WinOS_MidiIn.obj
 0001:00003af8       ??1Data@MidiIn_OpenHelper@@QEAA@XZ 0000000180004af8 f   PLATFORM_API_WinOS_MidiIn.obj
 0001:00003b40       ?MIDI_IN_PutMessage@@YAXPEAUHMIDIIN__@@I_K11@Z 0000000180004b40 f   PLATFORM_API_WinOS_MidiIn.obj
 0001:00003c00       ?ThreadProc@MidiIn_OpenHelper@@KAKPEAX@Z 0000000180004c00 f   PLATFORM_API_WinOS_MidiIn.obj
 0001:00003c60       ?getMidiInCaps@@YAHHPEAUtagMIDIINCAPSW@@PEAH@Z 0000000180004c60 f   PLATFORM_API_WinOS_MidiIn.obj
 0001:00003c8c       ?midiInOpen@MidiIn_OpenHelper@@SAIHPEAUtag_MidiDeviceHandle@@@Z 0000000180004c8c f   PLATFORM_API_WinOS_MidiIn.obj
 0001:00003d04       ?unprepareBuffers@@YAHPEAUtag_MidiDeviceHandle@@@Z 0000000180004d04 f   PLATFORM_API_WinOS_MidiIn.obj
 0001:00003d6c       MIDI_IN_CloseDevice        0000000180004d6c f   PLATFORM_API_WinOS_MidiIn.obj
 0001:00003dd8       MIDI_IN_GetDeviceDescription 0000000180004dd8 f   PLATFORM_API_WinOS_MidiIn.obj
 0001:00003dd8       MIDI_IN_GetDeviceVendor    0000000180004dd8 f   PLATFORM_API_WinOS_MidiIn.obj
 0001:00003dd8       MIDI_OUT_GetDeviceVendor   0000000180004dd8 f   PLATFORM_API_WinOS_MidiOut.obj
 0001:00003de0       MIDI_IN_GetDeviceName      0000000180004de0 f   PLATFORM_API_WinOS_MidiIn.obj
 0001:00003e60       MIDI_IN_GetDeviceVersion   0000000180004e60 f   PLATFORM_API_WinOS_MidiIn.obj
 0001:00003f00       MIDI_IN_GetErrorStr        0000000180004f00 f   PLATFORM_API_WinOS_MidiIn.obj
 0001:00003f2c       MIDI_IN_GetMessage         0000000180004f2c f   PLATFORM_API_WinOS_MidiIn.obj
 0001:00003f88       MIDI_IN_GetNumDevices      0000000180004f88 f   PLATFORM_API_WinOS_MidiIn.obj
 0001:00003f90       MIDI_IN_GetTimeStamp       0000000180004f90 f   PLATFORM_API_WinOS_MidiIn.obj
 0001:00003f90       MIDI_OUT_GetTimeStamp      0000000180004f90 f   PLATFORM_API_WinOS_MidiOut.obj
 0001:00003f98       MIDI_IN_OpenDevice         0000000180004f98 f   PLATFORM_API_WinOS_MidiIn.obj
 0001:000040e0       MIDI_IN_ReleaseMessage     00000001800050e0 f   PLATFORM_API_WinOS_MidiIn.obj
 0001:0000413c       MIDI_IN_StartDevice        000000018000513c f   PLATFORM_API_WinOS_MidiIn.obj
 0001:000041ac       MIDI_IN_StopDevice         00000001800051ac f   PLATFORM_API_WinOS_MidiIn.obj
 0001:00004218       __local_stdio_printf_options 0000000180005218 f i PLATFORM_API_WinOS_MidiIn.obj
 0001:00004220       snprintf                   0000000180005220 f i PLATFORM_API_WinOS_MidiIn.obj
 0001:00004278       MIDI_OUT_CloseDevice       0000000180005278 f   PLATFORM_API_WinOS_MidiOut.obj
 0001:00004338       MIDI_OUT_GetDeviceDescription 0000000180005338 f   PLATFORM_API_WinOS_MidiOut.obj
 0001:00004418       MIDI_OUT_GetDeviceName     0000000180005418 f   PLATFORM_API_WinOS_MidiOut.obj
 0001:00004498       MIDI_OUT_GetDeviceVersion  0000000180005498 f   PLATFORM_API_WinOS_MidiOut.obj
 0001:00004530       MIDI_OUT_GetErrorStr       0000000180005530 f   PLATFORM_API_WinOS_MidiOut.obj
 0001:0000455c       MIDI_OUT_GetNumDevices     000000018000555c f   PLATFORM_API_WinOS_MidiOut.obj
 0001:00004570       MIDI_OUT_OpenDevice        0000000180005570 f   PLATFORM_API_WinOS_MidiOut.obj
 0001:00004680       MIDI_OUT_SendLongMessage   0000000180005680 f   PLATFORM_API_WinOS_MidiOut.obj
 0001:000047f4       MIDI_OUT_SendShortMessage  00000001800057f4 f   PLATFORM_API_WinOS_MidiOut.obj
 0001:0000480c       freeLongBuffer             000000018000580c f   PLATFORM_API_WinOS_MidiOut.obj
 0001:0000488c       freeLongBuffers            000000018000588c f   PLATFORM_API_WinOS_MidiOut.obj
 0001:000048ec       getMidiOutCaps             00000001800058ec f   PLATFORM_API_WinOS_MidiOut.obj
 0001:0000492c       unprepareLongBuffers       000000018000592c f   PLATFORM_API_WinOS_MidiOut.obj
 0001:000049a0       PORT_Close                 00000001800059a0 f   PLATFORM_API_WinOS_Ports.obj
 0001:00004a38       PORT_GetControls           0000000180005a38 f   PLATFORM_API_WinOS_Ports.obj
 0001:00004cb4       PORT_GetFloatValue         0000000180005cb4 f   PLATFORM_API_WinOS_Ports.obj
 0001:00004d60       PORT_GetIntValue           0000000180005d60 f   PLATFORM_API_WinOS_Ports.obj
 0001:00004dac       PORT_GetPortCount          0000000180005dac f   PLATFORM_API_WinOS_Ports.obj
 0001:00004dbc       PORT_GetPortMixerCount     0000000180005dbc f   PLATFORM_API_WinOS_Ports.obj
 0001:00004dc4       PORT_GetPortMixerDescription 0000000180005dc4 f   PLATFORM_API_WinOS_Ports.obj
 0001:00004e78       PORT_GetPortName           0000000180005e78 f   PLATFORM_API_WinOS_Ports.obj
 0001:00004ed8       PORT_GetPortType           0000000180005ed8 f   PLATFORM_API_WinOS_Ports.obj
 0001:00004f0c       PORT_Open                  0000000180005f0c f   PLATFORM_API_WinOS_Ports.obj
 0001:000051cc       PORT_SetFloatValue         00000001800061cc f   PLATFORM_API_WinOS_Ports.obj
 0001:000052ac       PORT_SetIntValue           00000001800062ac f   PLATFORM_API_WinOS_Ports.obj
 0001:00005348       addAllControls             0000000180006348 f   PLATFORM_API_WinOS_Ports.obj
 0001:00005398       componentType2type         0000000180006398 f   PLATFORM_API_WinOS_Ports.obj
 0001:00005404       createLineControls         0000000180006404 f   PLATFORM_API_WinOS_Ports.obj
 0001:00005564       createMuxControl           0000000180006564 f   PLATFORM_API_WinOS_Ports.obj
 0001:000057a8       createPortControl          00000001800067a8 f   PLATFORM_API_WinOS_Ports.obj
 0001:0000596c       findDestLine               000000018000696c f   PLATFORM_API_WinOS_Ports.obj
 0001:000059a8       getControlCount            00000001800069a8 f   PLATFORM_API_WinOS_Ports.obj
 0001:00005a64       getControlInfo             0000000180006a64 f   PLATFORM_API_WinOS_Ports.obj
 0001:00005afc       getControlValue            0000000180006afc f   PLATFORM_API_WinOS_Ports.obj
 0001:00005b24       getDestinationCount        0000000180006b24 f   PLATFORM_API_WinOS_Ports.obj
 0001:00005b6c       getFakeBalance             0000000180006b6c f   PLATFORM_API_WinOS_Ports.obj
 0001:00005bcc       getMixerLineByDestination  0000000180006bcc f   PLATFORM_API_WinOS_Ports.obj
 0001:00005c0c       getMixerLineBySource       0000000180006c0c f   PLATFORM_API_WinOS_Ports.obj
 0001:00005c50       lineHasControls            0000000180006c50 f   PLATFORM_API_WinOS_Ports.obj
 0001:00005cd8       setControlValue            0000000180006cd8 f   PLATFORM_API_WinOS_Ports.obj
 0001:00005d00       setFakeVolume              0000000180006d00 f   PLATFORM_API_WinOS_Ports.obj
 0001:00005d70       MIDI_CreateLock            0000000180006d70 f   PLATFORM_API_WinOS_Util.obj
 0001:00005d98       MIDI_DestroyLock           0000000180006d98 f   PLATFORM_API_WinOS_Util.obj
 0001:00005dbc       MIDI_GetTimeStamp          0000000180006dbc f   PLATFORM_API_WinOS_Util.obj
 0001:00005dfc       MIDI_Lock                  0000000180006dfc f   PLATFORM_API_WinOS_Util.obj
 0001:00005e10       MIDI_SetStartTime          0000000180006e10 f   PLATFORM_API_WinOS_Util.obj
 0001:00005e30       MIDI_Unlock                0000000180006e30 f   PLATFORM_API_WinOS_Util.obj
 0001:00005e44       MIDI_WinCreateEmptyLongBufferQueue 0000000180006e44 f   PLATFORM_API_WinOS_Util.obj
 0001:00005e50       MIDI_WinCreateLongBufferQueue 0000000180006e50 f   PLATFORM_API_WinOS_Util.obj
 0001:00005f30       MIDI_WinDestroyLongBufferQueue 0000000180006f30 f   PLATFORM_API_WinOS_Util.obj
 0001:00005f68       Java_com_sun_media_sound_Platform_nIsBigEndian 0000000180006f68 f   Platform.obj
 0001:00005f70       GetInternalErrorStr        0000000180006f70 f   PlatformMidi.obj
 0001:00005fc0       MIDI_CreateQueue           0000000180006fc0 f   PlatformMidi.obj
 0001:00006010       MIDI_DestroyQueue          0000000180007010 f   PlatformMidi.obj
 0001:00006054       MIDI_IN_InternalGetErrorString 0000000180007054 f   PlatformMidi.obj
 0001:00006088       MIDI_OUT_InternalGetErrorString 0000000180007088 f   PlatformMidi.obj
 0001:000060bc       MIDI_QueueAddLong          00000001800070bc f   PlatformMidi.obj
 0001:000061a0       MIDI_QueueAddShort         00000001800071a0 f   PlatformMidi.obj
 0001:00006254       MIDI_QueueClear            0000000180007254 f   PlatformMidi.obj
 0001:00006284       MIDI_QueueRead             0000000180007284 f   PlatformMidi.obj
 0001:000062d8       MIDI_QueueRemove           00000001800072d8 f   PlatformMidi.obj
 0001:00006340       Java_com_sun_media_sound_PortMixer_nClose 0000000180007340 f   PortMixer.obj
 0001:00006358       Java_com_sun_media_sound_PortMixer_nControlGetFloatValue 0000000180007358 f   PortMixer.obj
 0001:00006374       Java_com_sun_media_sound_PortMixer_nControlGetIntValue 0000000180007374 f   PortMixer.obj
 0001:0000638c       Java_com_sun_media_sound_PortMixer_nControlSetFloatValue 000000018000738c f   PortMixer.obj
 0001:000063a8       Java_com_sun_media_sound_PortMixer_nControlSetIntValue 00000001800073a8 f   PortMixer.obj
 0001:000063c4       Java_com_sun_media_sound_PortMixer_nGetControls 00000001800073c4 f   PortMixer.obj
 0001:000064a4       Java_com_sun_media_sound_PortMixer_nGetPortCount 00000001800074a4 f   PortMixer.obj
 0001:000064bc       Java_com_sun_media_sound_PortMixer_nGetPortName 00000001800074bc f   PortMixer.obj
 0001:0000652c       Java_com_sun_media_sound_PortMixer_nGetPortType 000000018000752c f   PortMixer.obj
 0001:00006548       Java_com_sun_media_sound_PortMixer_nOpen 0000000180007548 f   PortMixer.obj
 0001:00006550       PORT_AddControl            0000000180007550 f   PortMixer.obj
 0001:00006588       PORT_NewBooleanControl     0000000180007588 f   PortMixer.obj
 0001:00006668       PORT_NewCompoundControl    0000000180007668 f   PortMixer.obj
 0001:000067a8       PORT_NewFloatControl       00000001800077a8 f   PortMixer.obj
 0001:00006950       Java_com_sun_media_sound_PortMixerProvider_nGetNumDevices 0000000180007950 f   PortMixerProvider.obj
 0001:00006958       Java_com_sun_media_sound_PortMixerProvider_nNewPortMixerInfo 0000000180007958 f   PortMixerProvider.obj
 0001:00006ab0       getPortMixerDescription    0000000180007ab0 f   PortMixerProvider.obj
 0001:00006b24       ThrowJavaMessageException  0000000180007b24 f   Utilities.obj
 0001:00006b5c       UTIL_IsBigEndianPlatform   0000000180007b5c f   Utilities.obj
 0001:00006b5c       __scrt_stub_for_is_c_termination_complete 0000000180007b5c f   MSVCRT:ucrt_stubs.obj
 0001:00006b5c       _is_c_termination_complete 0000000180007b5c f   MSVCRT:ucrt_stubs.obj
 0001:00006b5f       DirectSoundCreate          0000000180007b5f f   dsound:DSOUND.dll
 0001:00006b65       DirectSoundEnumerateA      0000000180007b65 f   dsound:DSOUND.dll
 0001:00006b6b       DirectSoundEnumerateW      0000000180007b6b f   dsound:DSOUND.dll
 0001:00006b71       DirectSoundCaptureCreate   0000000180007b71 f   dsound:DSOUND.dll
 0001:00006b77       DirectSoundCaptureEnumerateA 0000000180007b77 f   dsound:DSOUND.dll
 0001:00006b7d       DirectSoundCaptureEnumerateW 0000000180007b7d f   dsound:DSOUND.dll
 0001:00006b84       __GSHandlerCheck           0000000180007b84 f   MSVCRT:gshandler.obj
 0001:00006ba4       __GSHandlerCheckCommon     0000000180007ba4 f   MSVCRT:gshandler.obj
 0001:00006c10       __security_check_cookie    0000000180007c10 f   MSVCRT:amdsecgs.obj
 0001:00006c30       ??_U@YAPEAX_K@Z            0000000180007c30 f   MSVCRT:new_array.obj
 0001:00006c38       ??3@YAXPEAX_K@Z            0000000180007c38 f   MSVCRT:delete_scalar_size.obj
 0001:00006c38       ??_V@YAXPEAX@Z             0000000180007c38 f   MSVCRT:delete_array.obj
 0001:00006c40       __scrt_acquire_startup_lock 0000000180007c40 f   MSVCRT:utility.obj
 0001:00006c7c       __scrt_dllmain_after_initialize_c 0000000180007c7c f   MSVCRT:utility.obj
 0001:00006cb0       __scrt_dllmain_before_initialize_c 0000000180007cb0 f   MSVCRT:utility.obj
 0001:00006cc8       __scrt_dllmain_crt_thread_attach 0000000180007cc8 f   MSVCRT:utility.obj
 0001:00006cf0       __scrt_dllmain_crt_thread_detach 0000000180007cf0 f   MSVCRT:utility.obj
 0001:00006d08       __scrt_dllmain_exception_filter 0000000180007d08 f   MSVCRT:utility.obj
 0001:00006d68       __scrt_dllmain_uninitialize_c 0000000180007d68 f   MSVCRT:utility.obj
 0001:00006d98       __scrt_dllmain_uninitialize_critical 0000000180007d98 f   MSVCRT:utility.obj
 0001:00006dac       __scrt_initialize_crt      0000000180007dac f   MSVCRT:utility.obj
 0001:00006df8       __scrt_initialize_onexit_tables 0000000180007df8 f   MSVCRT:utility.obj
 0001:00006e84       __scrt_is_nonwritable_in_current_image 0000000180007e84 f   MSVCRT:utility.obj
 0001:00006f1c       __scrt_release_startup_lock 0000000180007f1c f   MSVCRT:utility.obj
 0001:00006f40       __scrt_uninitialize_crt    0000000180007f40 f   MSVCRT:utility.obj
 0001:00006f6c       _onexit                    0000000180007f6c f   MSVCRT:utility.obj
 0001:00006fa8       atexit                     0000000180007fa8 f   MSVCRT:utility.obj
 0001:000072e0       _DllMainCRTStartup         00000001800082e0 f   MSVCRT:dll_dllmain.obj
 0001:00007320       __raise_securityfailure    0000000180008320 f   MSVCRT:gs_report.obj
 0001:00007354       __report_gsfailure         0000000180008354 f   MSVCRT:gs_report.obj
 0001:0000749c       ??2@YAPEAX_K@Z             000000018000849c f   MSVCRT:new_scalar.obj
 0001:000074d8       ??3@YAXPEAX@Z              00000001800084d8 f   MSVCRT:delete_scalar.obj
 0001:000074e0       __isa_available_init       00000001800084e0 f   MSVCRT:cpu_disp.obj
 0001:0000768c       _get_startup_argv_mode     000000018000868c f   MSVCRT:argv_mode.obj
 0001:00007694       __scrt_is_ucrt_dll_in_use  0000000180008694 f   MSVCRT:ucrt_detection.obj
 0001:000076a0       __crt_debugger_hook        00000001800086a0 f   MSVCRT:utility_desktop.obj
 0001:000076a8       __scrt_fastfail            00000001800086a8 f   MSVCRT:utility_desktop.obj
 0001:000077f4       __security_init_cookie     00000001800087f4 f   MSVCRT:gs_support.obj
 0001:000078a0       DllMain                    00000001800088a0 f   MSVCRT:dll_dllmain_stub.obj
 0001:000078c4       ?__scrt_initialize_type_info@@YAXXZ 00000001800088c4 f   MSVCRT:tncleanup.obj
 0001:000078d4       ?__scrt_uninitialize_type_info@@YAXXZ 00000001800088d4 f   MSVCRT:tncleanup.obj
 0001:000078e0       __local_stdio_scanf_options 00000001800088e0 f i MSVCRT:default_local_stdio_options.obj
 0001:000078e8       __scrt_initialize_default_local_stdio_options 00000001800088e8 f   MSVCRT:default_local_stdio_options.obj
 0001:00007904       __scrt_get_dyn_tls_init_callback 0000000180008904 f   MSVCRT:dyn_tls_init.obj
 0001:0000790c       _RTC_Initialize            000000018000890c f   MSVCRT:initsect.obj
 0001:00007948       _RTC_Terminate             0000000180008948 f   MSVCRT:initsect.obj
 0001:00007984       ??0bad_alloc@std@@QEAA@AEBV01@@Z 0000000180008984 f i MSVCRT:throw_bad_alloc.obj
 0001:000079c0       ??0bad_alloc@std@@QEAA@XZ  00000001800089c0 f i MSVCRT:throw_bad_alloc.obj
 0001:000079e0       ??0bad_array_new_length@std@@QEAA@AEBV01@@Z 00000001800089e0 f i MSVCRT:throw_bad_alloc.obj
 0001:00007a1c       ??0bad_array_new_length@std@@QEAA@XZ 0000000180008a1c f i MSVCRT:throw_bad_alloc.obj
 0001:00007a3c       ??0exception@std@@QEAA@AEBV01@@Z 0000000180008a3c f i MSVCRT:throw_bad_alloc.obj
 0001:00007a70       ??1bad_alloc@std@@UEAA@XZ  0000000180008a70 f i MSVCRT:throw_bad_alloc.obj
 0001:00007a70       ??1bad_array_new_length@std@@UEAA@XZ 0000000180008a70 f i MSVCRT:throw_bad_alloc.obj
 0001:00007a84       ??_Ebad_alloc@std@@UEAAPEAXI@Z 0000000180008a84 f i MSVCRT:throw_bad_alloc.obj
 0001:00007a84       ??_Ebad_array_new_length@std@@UEAAPEAXI@Z 0000000180008a84 f i MSVCRT:throw_bad_alloc.obj
 0001:00007a84       ??_Eexception@std@@UEAAPEAXI@Z 0000000180008a84 f i MSVCRT:throw_bad_alloc.obj
 0001:00007a84       ??_Gbad_alloc@std@@UEAAPEAXI@Z 0000000180008a84 f i MSVCRT:throw_bad_alloc.obj
 0001:00007a84       ??_Gbad_array_new_length@std@@UEAAPEAXI@Z 0000000180008a84 f i MSVCRT:throw_bad_alloc.obj
 0001:00007a84       ??_Gexception@std@@UEAAPEAXI@Z 0000000180008a84 f i MSVCRT:throw_bad_alloc.obj
 0001:00007ac8       ?__scrt_throw_std_bad_alloc@@YAXXZ 0000000180008ac8 f   MSVCRT:throw_bad_alloc.obj
 0001:00007ae8       ?__scrt_throw_std_bad_array_new_length@@YAXXZ 0000000180008ae8 f   MSVCRT:throw_bad_alloc.obj
 0001:00007b08       ?what@exception@std@@UEBAPEBDXZ 0000000180008b08 f i MSVCRT:throw_bad_alloc.obj
 0001:00007b20       ??_Etype_info@@UEAAPEAXI@Z 0000000180008b20 f i MSVCRT:std_type_info_static.obj
 0001:00007b20       ??_Gtype_info@@UEAAPEAXI@Z 0000000180008b20 f i MSVCRT:std_type_info_static.obj
 0001:00007b4b       memcpy                     0000000180008b4b f   vcruntime:VCRUNTIME140.dll
 0001:00007b51       memset                     0000000180008b51 f   vcruntime:VCRUNTIME140.dll
 0001:00007b57       memcmp                     0000000180008b57 f   vcruntime:VCRUNTIME140.dll
 0001:00007b5d       __C_specific_handler       0000000180008b5d f   vcruntime:VCRUNTIME140.dll
 0001:00007b63       __std_type_info_destroy_list 0000000180008b63 f   vcruntime:VCRUNTIME140.dll
 0001:00007b69       __std_exception_copy       0000000180008b69 f   vcruntime:VCRUNTIME140.dll
 0001:00007b6f       __std_exception_destroy    0000000180008b6f f   vcruntime:VCRUNTIME140.dll
 0001:00007b75       _CxxThrowException         0000000180008b75 f   vcruntime:VCRUNTIME140.dll
 0001:00007b7b       free                       0000000180008b7b f   ucrt:api-ms-win-crt-heap-l1-1-0.dll
 0001:00007b81       malloc                     0000000180008b81 f   ucrt:api-ms-win-crt-heap-l1-1-0.dll
 0001:00007b87       strcpy                     0000000180008b87 f   ucrt:api-ms-win-crt-string-l1-1-0.dll
 0001:00007b8d       _seh_filter_dll            0000000180008b8d f   ucrt:api-ms-win-crt-runtime-l1-1-0.dll
 0001:00007b93       _configure_narrow_argv     0000000180008b93 f   ucrt:api-ms-win-crt-runtime-l1-1-0.dll
 0001:00007b99       _initialize_narrow_environment 0000000180008b99 f   ucrt:api-ms-win-crt-runtime-l1-1-0.dll
 0001:00007b9f       _initialize_onexit_table   0000000180008b9f f   ucrt:api-ms-win-crt-runtime-l1-1-0.dll
 0001:00007ba5       _register_onexit_function  0000000180008ba5 f   ucrt:api-ms-win-crt-runtime-l1-1-0.dll
 0001:00007bab       _execute_onexit_table      0000000180008bab f   ucrt:api-ms-win-crt-runtime-l1-1-0.dll
 0001:00007bb1       _crt_atexit                0000000180008bb1 f   ucrt:api-ms-win-crt-runtime-l1-1-0.dll
 0001:00007bb7       _cexit                     0000000180008bb7 f   ucrt:api-ms-win-crt-runtime-l1-1-0.dll
 0001:00007bbd       _initterm                  0000000180008bbd f   ucrt:api-ms-win-crt-runtime-l1-1-0.dll
 0001:00007bc3       _initterm_e                0000000180008bc3 f   ucrt:api-ms-win-crt-runtime-l1-1-0.dll
 0001:00007bc9       _callnewh                  0000000180008bc9 f   ucrt:api-ms-win-crt-heap-l1-1-0.dll
 0001:00007bd0       __acrt_initialize          0000000180008bd0 f   MSVCRT:ucrt_stubs.obj
 0001:00007bd0       __acrt_thread_attach       0000000180008bd0 f   MSVCRT:ucrt_stubs.obj
 0001:00007bd0       __acrt_thread_detach       0000000180008bd0 f   MSVCRT:ucrt_stubs.obj
 0001:00007bd0       __acrt_uninitialize        0000000180008bd0 f   MSVCRT:ucrt_stubs.obj
 0001:00007bd0       __acrt_uninitialize_critical 0000000180008bd0 f   MSVCRT:ucrt_stubs.obj
 0001:00007bd0       __scrt_stub_for_acrt_initialize 0000000180008bd0 f   MSVCRT:ucrt_stubs.obj
 0001:00007bd0       __scrt_stub_for_acrt_thread_attach 0000000180008bd0 f   MSVCRT:ucrt_stubs.obj
 0001:00007bd0       __scrt_stub_for_acrt_thread_detach 0000000180008bd0 f   MSVCRT:ucrt_stubs.obj
 0001:00007bd0       __scrt_stub_for_acrt_uninitialize 0000000180008bd0 f   MSVCRT:ucrt_stubs.obj
 0001:00007bd0       __scrt_stub_for_acrt_uninitialize_critical 0000000180008bd0 f   MSVCRT:ucrt_stubs.obj
 0001:00007bd0       __vcrt_initialize          0000000180008bd0 f   MSVCRT:ucrt_stubs.obj
 0001:00007bd0       __vcrt_thread_attach       0000000180008bd0 f   MSVCRT:ucrt_stubs.obj
 0001:00007bd0       __vcrt_thread_detach       0000000180008bd0 f   MSVCRT:ucrt_stubs.obj
 0001:00007bd0       __vcrt_uninitialize        0000000180008bd0 f   MSVCRT:ucrt_stubs.obj
 0001:00007bd0       __vcrt_uninitialize_critical 0000000180008bd0 f   MSVCRT:ucrt_stubs.obj
 0001:00007bf0       _guard_dispatch_icall_nop  0000000180008bf0 f   MSVCRT:guard_dispatch.obj
 0001:00007c10       _guard_xfg_dispatch_icall_nop 0000000180008c10 f   MSVCRT:guard_xfg_dispatch.obj
 0002:00000000       __imp_DirectSoundEnumerateA 0000000180009000     dsound:DSOUND.dll
 0002:00000008       __imp_DirectSoundEnumerateW 0000000180009008     dsound:DSOUND.dll
 0002:00000010       __imp_DirectSoundCaptureCreate 0000000180009010     dsound:DSOUND.dll
 0002:00000018       __imp_DirectSoundCaptureEnumerateA 0000000180009018     dsound:DSOUND.dll
 0002:00000020       __imp_DirectSoundCaptureEnumerateW 0000000180009020     dsound:DSOUND.dll
 0002:00000028       __imp_DirectSoundCreate    0000000180009028     dsound:DSOUND.dll
 0002:00000030       \177DSOUND_NULL_THUNK_DATA 0000000180009030     dsound:DSOUND.dll
 0002:00000038       __imp_InitializeSListHead  0000000180009038     kernel32:KERNEL32.dll
 0002:00000040       __imp_DisableThreadLibraryCalls 0000000180009040     kernel32:KERNEL32.dll
 0002:00000048       __imp_GetSystemTimeAsFileTime 0000000180009048     kernel32:KERNEL32.dll
 0002:00000050       __imp_GetCurrentThreadId   0000000180009050     kernel32:KERNEL32.dll
 0002:00000058       __imp_GetCurrentProcessId  0000000180009058     kernel32:KERNEL32.dll
 0002:00000060       __imp_QueryPerformanceCounter 0000000180009060     kernel32:KERNEL32.dll
 0002:00000068       __imp_IsDebuggerPresent    0000000180009068     kernel32:KERNEL32.dll
 0002:00000070       __imp_IsProcessorFeaturePresent 0000000180009070     kernel32:KERNEL32.dll
 0002:00000078       __imp_TerminateProcess     0000000180009078     kernel32:KERNEL32.dll
 0002:00000080       __imp_GetCurrentProcess    0000000180009080     kernel32:KERNEL32.dll
 0002:00000088       __imp_SetUnhandledExceptionFilter 0000000180009088     kernel32:KERNEL32.dll
 0002:00000090       __imp_UnhandledExceptionFilter 0000000180009090     kernel32:KERNEL32.dll
 0002:00000098       __imp_RtlVirtualUnwind     0000000180009098     kernel32:KERNEL32.dll
 0002:000000a0       __imp_RtlLookupFunctionEntry 00000001800090a0     kernel32:KERNEL32.dll
 0002:000000a8       __imp_RtlCaptureContext    00000001800090a8     kernel32:KERNEL32.dll
 0002:000000b0       __imp_DeleteCriticalSection 00000001800090b0     kernel32:KERNEL32.dll
 0002:000000b8       __imp_Sleep                00000001800090b8     kernel32:KERNEL32.dll
 0002:000000c0       __imp_CreateThread         00000001800090c0     kernel32:KERNEL32.dll
 0002:000000c8       __imp_CreateEventA         00000001800090c8     kernel32:KERNEL32.dll
 0002:000000d0       __imp_WaitForSingleObject  00000001800090d0     kernel32:KERNEL32.dll
 0002:000000d8       __imp_SetEvent             00000001800090d8     kernel32:KERNEL32.dll
 0002:000000e0       __imp_LeaveCriticalSection 00000001800090e0     kernel32:KERNEL32.dll
 0002:000000e8       __imp_EnterCriticalSection 00000001800090e8     kernel32:KERNEL32.dll
 0002:000000f0       __imp_InitializeCriticalSection 00000001800090f0     kernel32:KERNEL32.dll
 0002:000000f8       __imp_CloseHandle          00000001800090f8     kernel32:KERNEL32.dll
 0002:00000100       __imp_WideCharToMultiByte  0000000180009100     kernel32:KERNEL32.dll
 0002:00000108       \177KERNEL32_NULL_THUNK_DATA 0000000180009108     kernel32:KERNEL32.dll
 0002:00000110       __imp_GetDesktopWindow     0000000180009110     user32:USER32.dll
 0002:00000118       __imp_GetForegroundWindow  0000000180009118     user32:USER32.dll
 0002:00000120       \177USER32_NULL_THUNK_DATA 0000000180009120     user32:USER32.dll
 0002:00000128       __imp___C_specific_handler 0000000180009128     vcruntime:VCRUNTIME140.dll
 0002:00000130       __imp_memset               0000000180009130     vcruntime:VCRUNTIME140.dll
 0002:00000138       __imp_memcmp               0000000180009138     vcruntime:VCRUNTIME140.dll
 0002:00000140       __imp__CxxThrowException   0000000180009140     vcruntime:VCRUNTIME140.dll
 0002:00000148       __imp___std_exception_destroy 0000000180009148     vcruntime:VCRUNTIME140.dll
 0002:00000150       __imp___std_exception_copy 0000000180009150     vcruntime:VCRUNTIME140.dll
 0002:00000158       __imp_memcpy               0000000180009158     vcruntime:VCRUNTIME140.dll
 0002:00000160       __imp___std_type_info_destroy_list 0000000180009160     vcruntime:VCRUNTIME140.dll
 0002:00000168       \177VCRUNTIME140_NULL_THUNK_DATA 0000000180009168     vcruntime:VCRUNTIME140.dll
 0002:00000170       __imp_timeEndPeriod        0000000180009170     winmm:WINMM.dll
 0002:00000178       __imp_timeBeginPeriod      0000000180009178     winmm:WINMM.dll
 0002:00000180       __imp_midiOutReset         0000000180009180     winmm:WINMM.dll
 0002:00000188       __imp_midiOutLongMsg       0000000180009188     winmm:WINMM.dll
 0002:00000190       __imp_midiOutShortMsg      0000000180009190     winmm:WINMM.dll
 0002:00000198       __imp_midiOutUnprepareHeader 0000000180009198     winmm:WINMM.dll
 0002:000001a0       __imp_midiOutPrepareHeader 00000001800091a0     winmm:WINMM.dll
 0002:000001a8       __imp_midiOutClose         00000001800091a8     winmm:WINMM.dll
 0002:000001b0       __imp_mixerGetDevCapsW     00000001800091b0     winmm:WINMM.dll
 0002:000001b8       __imp_midiOutGetErrorTextA 00000001800091b8     winmm:WINMM.dll
 0002:000001c0       __imp_midiOutGetDevCapsW   00000001800091c0     winmm:WINMM.dll
 0002:000001c8       __imp_midiOutGetNumDevs    00000001800091c8     winmm:WINMM.dll
 0002:000001d0       __imp_midiInReset          00000001800091d0     winmm:WINMM.dll
 0002:000001d8       __imp_midiInStop           00000001800091d8     winmm:WINMM.dll
 0002:000001e0       __imp_midiInStart          00000001800091e0     winmm:WINMM.dll
 0002:000001e8       __imp_midiInAddBuffer      00000001800091e8     winmm:WINMM.dll
 0002:000001f0       __imp_midiInUnprepareHeader 00000001800091f0     winmm:WINMM.dll
 0002:000001f8       __imp_midiInPrepareHeader  00000001800091f8     winmm:WINMM.dll
 0002:00000200       __imp_midiInClose          0000000180009200     winmm:WINMM.dll
 0002:00000208       __imp_midiInOpen           0000000180009208     winmm:WINMM.dll
 0002:00000210       __imp_midiInGetErrorTextA  0000000180009210     winmm:WINMM.dll
 0002:00000218       __imp_midiInGetDevCapsW    0000000180009218     winmm:WINMM.dll
 0002:00000220       __imp_midiInGetNumDevs     0000000180009220     winmm:WINMM.dll
 0002:00000228       __imp_timeGetTime          0000000180009228     winmm:WINMM.dll
 0002:00000230       __imp_mixerOpen            0000000180009230     winmm:WINMM.dll
 0002:00000238       __imp_mixerClose           0000000180009238     winmm:WINMM.dll
 0002:00000240       __imp_mixerGetNumDevs      0000000180009240     winmm:WINMM.dll
 0002:00000248       __imp_mixerSetControlDetails 0000000180009248     winmm:WINMM.dll
 0002:00000250       __imp_mixerGetControlDetailsA 0000000180009250     winmm:WINMM.dll
 0002:00000258       __imp_mixerGetLineControlsA 0000000180009258     winmm:WINMM.dll
 0002:00000260       __imp_midiOutOpen          0000000180009260     winmm:WINMM.dll
 0002:00000268       __imp_mixerGetLineInfoA    0000000180009268     winmm:WINMM.dll
 0002:00000270       \177WINMM_NULL_THUNK_DATA  0000000180009270     winmm:WINMM.dll
 0002:00000278       __imp_malloc               0000000180009278     ucrt:api-ms-win-crt-heap-l1-1-0.dll
 0002:00000280       __imp_free                 0000000180009280     ucrt:api-ms-win-crt-heap-l1-1-0.dll
 0002:00000288       __imp__callnewh            0000000180009288     ucrt:api-ms-win-crt-heap-l1-1-0.dll
 0002:00000290       \177api-ms-win-crt-heap-l1-1-0_NULL_THUNK_DATA 0000000180009290     ucrt:api-ms-win-crt-heap-l1-1-0.dll
 0002:00000298       __imp__register_onexit_function 0000000180009298     ucrt:api-ms-win-crt-runtime-l1-1-0.dll
 0002:000002a0       __imp__initterm_e          00000001800092a0     ucrt:api-ms-win-crt-runtime-l1-1-0.dll
 0002:000002a8       __imp__initterm            00000001800092a8     ucrt:api-ms-win-crt-runtime-l1-1-0.dll
 0002:000002b0       __imp__seh_filter_dll      00000001800092b0     ucrt:api-ms-win-crt-runtime-l1-1-0.dll
 0002:000002b8       __imp__configure_narrow_argv 00000001800092b8     ucrt:api-ms-win-crt-runtime-l1-1-0.dll
 0002:000002c0       __imp__initialize_narrow_environment 00000001800092c0     ucrt:api-ms-win-crt-runtime-l1-1-0.dll
 0002:000002c8       __imp__initialize_onexit_table 00000001800092c8     ucrt:api-ms-win-crt-runtime-l1-1-0.dll
 0002:000002d0       __imp__execute_onexit_table 00000001800092d0     ucrt:api-ms-win-crt-runtime-l1-1-0.dll
 0002:000002d8       __imp__crt_atexit          00000001800092d8     ucrt:api-ms-win-crt-runtime-l1-1-0.dll
 0002:000002e0       __imp__cexit               00000001800092e0     ucrt:api-ms-win-crt-runtime-l1-1-0.dll
 0002:000002e8       \177api-ms-win-crt-runtime-l1-1-0_NULL_THUNK_DATA 00000001800092e8     ucrt:api-ms-win-crt-runtime-l1-1-0.dll
 0002:000002f0       __imp___stdio_common_vsprintf 00000001800092f0     ucrt:api-ms-win-crt-stdio-l1-1-0.dll
 0002:000002f8       \177api-ms-win-crt-stdio-l1-1-0_NULL_THUNK_DATA 00000001800092f8     ucrt:api-ms-win-crt-stdio-l1-1-0.dll
 0002:00000300       __imp_strcpy               0000000180009300     ucrt:api-ms-win-crt-string-l1-1-0.dll
 0002:00000308       __imp_strncpy              0000000180009308     ucrt:api-ms-win-crt-string-l1-1-0.dll
 0002:00000310       \177api-ms-win-crt-string-l1-1-0_NULL_THUNK_DATA 0000000180009310     ucrt:api-ms-win-crt-string-l1-1-0.dll
 0002:00000318       __imp_CoInitialize         0000000180009318     ole32:ole32.dll
 0002:00000320       __imp_CoUninitialize       0000000180009320     ole32:ole32.dll
 0002:00000328       \177ole32_NULL_THUNK_DATA  0000000180009328     ole32:ole32.dll
 0002:00000330       __guard_check_icall_fptr   0000000180009330     MSVCRT:guard_support.obj
 0002:00000338       __guard_xfg_check_icall_fptr 0000000180009338     MSVCRT:guard_support.obj
 0002:00000340       __guard_dispatch_icall_fptr 0000000180009340     MSVCRT:guard_support.obj
 0002:00000348       __guard_xfg_dispatch_icall_fptr 0000000180009348     MSVCRT:guard_support.obj
 0002:00000350       __guard_xfg_table_dispatch_icall_fptr 0000000180009350     MSVCRT:guard_support.obj
 0002:00000358       __castguard_check_failure_os_handled_fptr 0000000180009358     MSVCRT:guard_support.obj
 0002:00000360       __guard_memcpy_fptr        0000000180009360     vcruntime:softmemtag.obj
 0002:00000368       __xc_a                     0000000180009368     MSVCRT:initializers.obj
 0002:00000380       __xc_z                     0000000180009380     MSVCRT:initializers.obj
 0002:00000388       __xi_a                     0000000180009388     MSVCRT:initializers.obj
 0002:00000390       __xi_z                     0000000180009390     MSVCRT:initializers.obj
 0002:00000398       __xp_a                     0000000180009398     MSVCRT:initializers.obj
 0002:000003a0       __xp_z                     00000001800093a0     MSVCRT:initializers.obj
 0002:000003a8       __xt_a                     00000001800093a8     MSVCRT:initializers.obj
 0002:000003b0       __xt_z                     00000001800093b0     MSVCRT:initializers.obj
 0002:000003c0       ??_C@_0BN@PPKEDFNA@?$CILjava?1util?1Vector?$DLIIIFIZZ?$CJV@ 00000001800093c0     DirectAudioDevice.obj
 0002:000003e0       ??_C@_09OBBPPKHG@addFormat@ 00000001800093e0     DirectAudioDevice.obj
 0002:000003ec       __real@3f800000            00000001800093ec     DirectAudioDevice.obj
 0002:000003f0       __real@3f847ae147ae147b    00000001800093f0     DirectAudioDevice.obj
 0002:00000400       __xmm@7fffffff7fffffff7fffffff7fffffff 0000000180009400     DirectAudioDevice.obj
 0002:00000410       ??_C@_0N@FMCAPCBL@Unknown?5Name@ 0000000180009410     DirectAudioDeviceProvider.obj
 0002:00000420       ??_C@_0P@JELLBOOJ@Unknown?5Vendor@ 0000000180009420     DirectAudioDeviceProvider.obj
 0002:00000430       ??_C@_0BE@GEPKBKKC@Unknown?5Description@ 0000000180009430     DirectAudioDeviceProvider.obj
 0002:00000448       ??_C@_0BA@LFHNEBGG@Unknown?5Version@ 0000000180009448     DirectAudioDeviceProvider.obj
 0002:00000460       ??_C@_0EE@IPKJIHIL@com?1sun?1media?1sound?1DirectAudio@ 0000000180009460     DirectAudioDeviceProvider.obj
 0002:000004b0       ??_C@_0EP@IBGEIIFD@?$CIIIILjava?1lang?1String?$DLLjava?1lan@ 00000001800094b0     DirectAudioDeviceProvider.obj
 0002:00000500       ??_C@_06FALKBLGB@?$DMinit?$DO@ 0000000180009500     DirectAudioDeviceProvider.obj
 0002:00000508       ??_C@_0CK@BNIEGIBB@javax?1sound?1midi?1MidiUnavailabl@ 0000000180009508     MidiInDevice.obj
 0002:00000534       ??_C@_05NPPFNMNL@?$CIIJ?$CJV@ 0000000180009534     MidiInDevice.obj
 0002:00000540       ??_C@_0BF@LEBFAHIB@callbackShortMessage@ 0000000180009540     MidiInDevice.obj
 0002:00000558       ??_C@_06PFGPJLID@?$CI?$FLBJ?$CJV@ 0000000180009558     MidiInDevice.obj
 0002:00000560       ??_C@_0BE@CLHHHCK@callbackLongMessage@ 0000000180009560     MidiInDevice.obj
 0002:00000578       ??_C@_0N@JNOBNNBP@Unknown?5name@ 0000000180009578     MidiInDeviceProvider.obj
 0002:00000588       ??_C@_0P@FLAGCHHF@Unknown?5vendor@ 0000000180009588     MidiInDeviceProvider.obj
 0002:00000598       ??_C@_0BF@LIAFPILD@No?5details?5available@ 0000000180009598     MidiInDeviceProvider.obj
 0002:000005b0       ??_C@_0BA@EMALCDDA@Unknown?5version@ 00000001800095b0     MidiInDeviceProvider.obj
 0002:000005c0       ??_C@_0BF@HPHHCMEI@DirectSound?5Playback@ 00000001800095c0     PLATFORM_API_WinOS_DirectSound.obj
 0002:000005d8       ??_C@_0BE@OBEMNMJC@DirectSound?5Capture@ 00000001800095d8     PLATFORM_API_WinOS_DirectSound.obj
 0002:000005ec       ??_C@_05KBEOJPB@?$CFd?4?$CFd@ 00000001800095ec     PLATFORM_API_WinOS_MidiIn.obj
 0002:000005f8       ??_C@_0BD@GIDICAOP@External?5MIDI?5Port@ 00000001800095f8     PLATFORM_API_WinOS_MidiOut.obj
 0002:00000610       ??_C@_0CB@BKPHBOPD@Internal?5square?5wave?5synthesize@ 0000000180009610     PLATFORM_API_WinOS_MidiOut.obj
 0002:00000638       ??_C@_0BI@BENILECD@Internal?5FM?5synthesizer@ 0000000180009638     PLATFORM_API_WinOS_MidiOut.obj
 0002:00000650       ??_C@_0BP@HFJPHHGA@Internal?5synthesizer?5?$CIgeneric?$CJ@ 0000000180009650     PLATFORM_API_WinOS_MidiOut.obj
 0002:00000670       ??_C@_0BE@GKHJJDH@Windows?5MIDI_MAPPER@ 0000000180009670     PLATFORM_API_WinOS_MidiOut.obj
 0002:00000688       ??_C@_0BO@JHOFOEDM@Internal?5software?5synthesizer@ 0000000180009688     PLATFORM_API_WinOS_MidiOut.obj
 0002:000006a8       ??_C@_0L@CPKCBHCN@Port?5Mixer@ 00000001800096a8     PLATFORM_API_WinOS_Ports.obj
 0002:000006b3       ??_C@_00CNPNBAHC@@         00000001800096b3     PLATFORM_API_WinOS_Ports.obj
 0002:000006b4       __real@3f000000            00000001800096b4     PLATFORM_API_WinOS_Ports.obj
 0002:000006b8       __real@40000000            00000001800096b8     PLATFORM_API_WinOS_Ports.obj
 0002:000006bc       __real@bf800000            00000001800096bc     PLATFORM_API_WinOS_Ports.obj
 0002:000006c0       ??_C@_0BG@PNPJGPKL@feature?5not?5supported@ 00000001800096c0     PlatformMidi.obj
 0002:000006d8       ??_C@_0BC@GOGOPKAK@invalid?5device?5ID@ 00000001800096d8     PlatformMidi.obj
 0002:000006f0       ??_C@_0BP@CMLKCPDD@internal?5error?3?5invalid?5handle@ 00000001800096f0     PlatformMidi.obj
 0002:00000710       ??_C@_0O@BNNCBLEN@out?5of?5memory@ 0000000180009710     PlatformMidi.obj
 0002:00000720       ??_C@_0CH@PANCBAOC@com?1sun?1media?1sound?1PortMixer$B@ 0000000180009720     PortMixer.obj
 0002:00000748       ??_C@_0BH@DOGHFNPN@?$CIJLjava?1lang?1String?$DL?$CJV@ 0000000180009748     PortMixer.obj
 0002:00000760       ??_C@_04IOCNJLNK@Mute@     0000000180009760     PortMixer.obj
 0002:00000768       ??_C@_06HJGPBJLE@Select@   0000000180009768     PortMixer.obj
 0002:00000770       ??_C@_0CH@ECCNHGI@com?1sun?1media?1sound?1PortMixer$C@ 0000000180009770     PortMixer.obj
 0002:00000798       ??_C@_0DE@OMOINGJL@?$CILjava?1lang?1String?$DL?$FLLjavax?1soun@ 0000000180009798     PortMixer.obj
 0002:000007d0       ??_C@_0BM@GDMEENBL@javax?1sound?1sampled?1Control@ 00000001800097d0     PortMixer.obj
 0002:000007f0       ??_C@_0CI@OPKAAKLF@com?1sun?1media?1sound?1PortMixer$F@ 00000001800097f0     PortMixer.obj
 0002:00000818       ??_C@_0CM@PEFBHGMP@?$CIJLjava?1lang?1String?$DLFFFLjava?1la@ 0000000180009818     PortMixer.obj
 0002:00000848       ??_C@_0BL@HJNALIL@?$CIJIFFFLjava?1lang?1String?$DL?$CJV@ 0000000180009848     PortMixer.obj
 0002:00000868       ??_C@_0BG@JLFLBLJI@?$CILjava?1lang?1Object?$DL?$CJV@ 0000000180009868     PortMixer.obj
 0002:00000880       ??_C@_0L@MNLDOJKN@addElement@ 0000000180009880     PortMixer.obj
 0002:00000890       ??_C@_0DE@HOKEHCEP@com?1sun?1media?1sound?1PortMixerPr@ 0000000180009890     PortMixerProvider.obj
 0002:000008d0       ??_C@_0EN@JGCFGEEO@?$CIILjava?1lang?1String?$DLLjava?1lang?1@ 00000001800098d0     PortMixerProvider.obj
 0002:00000920       __xmm@ffffffffffffffffffffffffffffffff 0000000180009920     MSVCRT:utility.obj
 0002:00000930       _pDefaultRawDllMain        0000000180009930     MSVCRT:dll_dllmain.obj
 0002:00000930       _pRawDllMain               0000000180009930     MSVCRT:dll_dllmain.obj
 0002:00000950       ??_7exception@std@@6B@     0000000180009950     MSVCRT:throw_bad_alloc.obj
 0002:00000960       ??_C@_0BC@EOODALEL@Unknown?5exception@ 0000000180009960     MSVCRT:throw_bad_alloc.obj
 0002:00000980       ??_7bad_alloc@std@@6B@     0000000180009980     MSVCRT:throw_bad_alloc.obj
 0002:00000990       ??_C@_0P@GHFPNOJB@bad?5allocation@ 0000000180009990     MSVCRT:throw_bad_alloc.obj
 0002:000009a8       ??_7bad_array_new_length@std@@6B@ 00000001800099a8     MSVCRT:throw_bad_alloc.obj
 0002:000009b8       ??_C@_0BF@KINCDENJ@bad?5array?5new?5length@ 00000001800099b8     MSVCRT:throw_bad_alloc.obj
 0002:000009d8       ??_7type_info@@6B@         00000001800099d8     MSVCRT:std_type_info_static.obj
 0002:000009e0       _load_config_used          00000001800099e0     MSVCRT:loadcfg.obj
 0002:00000c00       ??_R4exception@std@@6B@    0000000180009c00     MSVCRT:throw_bad_alloc.obj
 0002:00000c28       ??_R3exception@std@@8      0000000180009c28     MSVCRT:throw_bad_alloc.obj
 0002:00000c40       ??_R2exception@std@@8      0000000180009c40     MSVCRT:throw_bad_alloc.obj
 0002:00000c50       ??_R1A@?0A@EA@exception@std@@8 0000000180009c50     MSVCRT:throw_bad_alloc.obj
 0002:00000c78       ??_R4bad_alloc@std@@6B@    0000000180009c78     MSVCRT:throw_bad_alloc.obj
 0002:00000ca0       ??_R3bad_alloc@std@@8      0000000180009ca0     MSVCRT:throw_bad_alloc.obj
 0002:00000cb8       ??_R2bad_alloc@std@@8      0000000180009cb8     MSVCRT:throw_bad_alloc.obj
 0002:00000cd0       ??_R1A@?0A@EA@bad_alloc@std@@8 0000000180009cd0     MSVCRT:throw_bad_alloc.obj
 0002:00000cf8       ??_R4bad_array_new_length@std@@6B@ 0000000180009cf8     MSVCRT:throw_bad_alloc.obj
 0002:00000d20       ??_R3bad_array_new_length@std@@8 0000000180009d20     MSVCRT:throw_bad_alloc.obj
 0002:00000d38       ??_R2bad_array_new_length@std@@8 0000000180009d38     MSVCRT:throw_bad_alloc.obj
 0002:00000d58       ??_R1A@?0A@EA@bad_array_new_length@std@@8 0000000180009d58     MSVCRT:throw_bad_alloc.obj
 0002:00000d80       ??_R4type_info@@6B@        0000000180009d80     MSVCRT:std_type_info_static.obj
 0002:00000da8       ??_R3type_info@@8          0000000180009da8     MSVCRT:std_type_info_static.obj
 0002:00000dc0       ??_R2type_info@@8          0000000180009dc0     MSVCRT:std_type_info_static.obj
 0002:00000dd0       ??_R1A@?0A@EA@type_info@@8 0000000180009dd0     MSVCRT:std_type_info_static.obj
 0002:00000df4       __volatile_metadata        0000000180009df4     <linker-defined>
 0002:00001240       __rtc_iaa                  000000018000a240     MSVCRT:initsect.obj
 0002:00001248       __rtc_izz                  000000018000a248     MSVCRT:initsect.obj
 0002:00001250       __rtc_taa                  000000018000a250     MSVCRT:initsect.obj
 0002:00001258       __rtc_tzz                  000000018000a258     MSVCRT:initsect.obj
 0002:00001810       _TI2?AVbad_alloc@std@@     000000018000a810     MSVCRT:throw_bad_alloc.obj
 0002:00001830       _CTA2?AVbad_alloc@std@@    000000018000a830     MSVCRT:throw_bad_alloc.obj
 0002:00001848       _CT??_R0?AVbad_alloc@std@@@8??0bad_alloc@std@@QEAA@AEBV01@@Z24 000000018000a848     MSVCRT:throw_bad_alloc.obj
 0002:00001870       _CT??_R0?AVexception@std@@@8??0exception@std@@QEAA@AEBV01@@Z24 000000018000a870     MSVCRT:throw_bad_alloc.obj
 0002:00001898       _TI3?AVbad_array_new_length@std@@ 000000018000a898     MSVCRT:throw_bad_alloc.obj
 0002:000018b8       _CTA3?AVbad_array_new_length@std@@ 000000018000a8b8     MSVCRT:throw_bad_alloc.obj
 0002:000018d8       _CT??_R0?AVbad_array_new_length@std@@@8??0bad_array_new_length@std@@QEAA@AEBV01@@Z24 000000018000a8d8     MSVCRT:throw_bad_alloc.obj
 0002:000025ec       __IMPORT_DESCRIPTOR_DSOUND 000000018000b5ec     dsound:DSOUND.dll
 0002:00002600       __IMPORT_DESCRIPTOR_WINMM  000000018000b600     winmm:WINMM.dll
 0002:00002614       __IMPORT_DESCRIPTOR_USER32 000000018000b614     user32:USER32.dll
 0002:00002628       __IMPORT_DESCRIPTOR_ole32  000000018000b628     ole32:ole32.dll
 0002:0000263c       __IMPORT_DESCRIPTOR_KERNEL32 000000018000b63c     kernel32:KERNEL32.dll
 0002:00002650       __IMPORT_DESCRIPTOR_VCRUNTIME140 000000018000b650     vcruntime:VCRUNTIME140.dll
 0002:00002664       __IMPORT_DESCRIPTOR_api-ms-win-crt-heap-l1-1-0 000000018000b664     ucrt:api-ms-win-crt-heap-l1-1-0.dll
 0002:00002678       __IMPORT_DESCRIPTOR_api-ms-win-crt-string-l1-1-0 000000018000b678     ucrt:api-ms-win-crt-string-l1-1-0.dll
 0002:0000268c       __IMPORT_DESCRIPTOR_api-ms-win-crt-stdio-l1-1-0 000000018000b68c     ucrt:api-ms-win-crt-stdio-l1-1-0.dll
 0002:000026a0       __IMPORT_DESCRIPTOR_api-ms-win-crt-runtime-l1-1-0 000000018000b6a0     ucrt:api-ms-win-crt-runtime-l1-1-0.dll
 0002:000026b4       __NULL_IMPORT_DESCRIPTOR   000000018000b6b4     dsound:DSOUND.dll
 0003:00000018       _fltused                   000000018000d018     MSVCRT:fltused.obj
 0003:00000020       __security_cookie_complement 000000018000d020     MSVCRT:gs_cookie.obj
 0003:00000028       __security_cookie          000000018000d028     MSVCRT:gs_cookie.obj
 0003:00000030       __scrt_native_dllmain_reason 000000018000d030     MSVCRT:utility.obj
 0003:00000038       __isa_available            000000018000d038     MSVCRT:cpu_disp.obj
 0003:0000003c       __isa_enabled              000000018000d03c     MSVCRT:cpu_disp.obj
 0003:00000040       __memset_fast_string_threshold 000000018000d040     MSVCRT:cpu_disp.obj
 0003:00000048       __memset_nt_threshold      000000018000d048     MSVCRT:cpu_disp.obj
 0003:00000050       __scrt_ucrt_dll_is_in_use  000000018000d050     MSVCRT:ucrt_stubs.obj
 0003:00000058       ??_R0?AVbad_alloc@std@@@8  000000018000d058     MSVCRT:throw_bad_alloc.obj
 0003:00000080       ??_R0?AVexception@std@@@8  000000018000d080     MSVCRT:throw_bad_alloc.obj
 0003:000000a8       ??_R0?AVbad_array_new_length@std@@@8 000000018000d0a8     MSVCRT:throw_bad_alloc.obj
 0003:000000d8       ??_R0?AVtype_info@@@8      000000018000d0d8     MSVCRT:std_type_info_static.obj
 0003:00000100       ?data@DS_StartBufferHelper@@1VData@1@A 000000018000d100     PLATFORM_API_WinOS_DirectSound.obj
 0003:00000ad0       ?_OptionsStorage@?1??__local_stdio_printf_options@@9@4_KA 000000018000dad0     PLATFORM_API_WinOS_MidiIn.obj
 0003:00000ae0       ?data@MidiIn_OpenHelper@@1VData@1@A 000000018000dae0     PLATFORM_API_WinOS_MidiIn.obj
 0003:00000cc8       __scrt_current_native_startup_state 000000018000dcc8     MSVCRT:utility.obj
 0003:00000cd0       __scrt_native_startup_lock 000000018000dcd0     MSVCRT:utility.obj
 0003:00001290       __favor                    000000018000e290     MSVCRT:cpu_disp.obj
 0003:00001294       __scrt_debugger_hook_flag  000000018000e294     MSVCRT:utility_desktop.obj
 0003:000012a0       ?__type_info_root_node@@3U__type_info_node@@A 000000018000e2a0     MSVCRT:tncleanup.obj
 0003:000012b0       ?_OptionsStorage@?1??__local_stdio_scanf_options@@9@4_KA 000000018000e2b0     MSVCRT:default_local_stdio_options.obj
 0003:000012b8       __dyn_tls_init_callback    000000018000e2b8     <common>

 entry point at        0001:000072e0

 Static symbols

 0000:fffee000       .debug$S                   0000000180000000     jsound.exp
 0000:fffee000       .debug$S                   0000000180000000     vcruntime:VCRUNTIME140.dll
 0000:fffee000       .debug$S                   0000000180000000     vcruntime:VCRUNTIME140.dll
 0000:fffee000       .debug$S                   0000000180000000     vcruntime:VCRUNTIME140.dll
 0000:fffee000       .debug$S                   0000000180000000     vcruntime:VCRUNTIME140.dll
 0000:fffee000       .debug$S                   0000000180000000     vcruntime:VCRUNTIME140.dll
 0000:fffee000       .debug$S                   0000000180000000     vcruntime:VCRUNTIME140.dll
 0000:fffee000       .debug$S                   0000000180000000     vcruntime:VCRUNTIME140.dll
 0000:fffee000       .debug$S                   0000000180000000     vcruntime:VCRUNTIME140.dll
 0000:fffee000       .debug$S                   0000000180000000     vcruntime:VCRUNTIME140.dll
 0000:fffee000       .debug$S                   0000000180000000     vcruntime:VCRUNTIME140.dll
 0000:fffee000       .debug$S                   0000000180000000     ucrt:api-ms-win-crt-heap-l1-1-0.dll
 0000:fffee000       .debug$S                   0000000180000000     ucrt:api-ms-win-crt-heap-l1-1-0.dll
 0000:fffee000       .debug$S                   0000000180000000     ucrt:api-ms-win-crt-heap-l1-1-0.dll
 0000:fffee000       .debug$S                   0000000180000000     ucrt:api-ms-win-crt-runtime-l1-1-0.dll
 0000:fffee000       .debug$S                   0000000180000000     ucrt:api-ms-win-crt-runtime-l1-1-0.dll
 0000:fffee000       .debug$S                   0000000180000000     ucrt:api-ms-win-crt-runtime-l1-1-0.dll
 0000:fffee000       .debug$S                   0000000180000000     ucrt:api-ms-win-crt-runtime-l1-1-0.dll
 0000:fffee000       .debug$S                   0000000180000000     ucrt:api-ms-win-crt-runtime-l1-1-0.dll
 0000:fffee000       .debug$S                   0000000180000000     ucrt:api-ms-win-crt-runtime-l1-1-0.dll
 0000:fffee000       .debug$S                   0000000180000000     ucrt:api-ms-win-crt-runtime-l1-1-0.dll
 0000:fffee000       .debug$S                   0000000180000000     ucrt:api-ms-win-crt-runtime-l1-1-0.dll
 0000:fffee000       .debug$S                   0000000180000000     ucrt:api-ms-win-crt-runtime-l1-1-0.dll
 0000:fffee000       .debug$S                   0000000180000000     ucrt:api-ms-win-crt-runtime-l1-1-0.dll
 0000:fffee000       .debug$S                   0000000180000000     ucrt:api-ms-win-crt-runtime-l1-1-0.dll
 0000:fffee000       .debug$S                   0000000180000000     ucrt:api-ms-win-crt-runtime-l1-1-0.dll
 0000:fffee000       .debug$S                   0000000180000000     ucrt:api-ms-win-crt-stdio-l1-1-0.dll
 0000:fffee000       .debug$S                   0000000180000000     ucrt:api-ms-win-crt-string-l1-1-0.dll
 0000:fffee000       .debug$S                   0000000180000000     ucrt:api-ms-win-crt-string-l1-1-0.dll
 0000:fffee000       .debug$S                   0000000180000000     dsound:DSOUND.dll
 0000:fffee000       .debug$S                   0000000180000000     dsound:DSOUND.dll
 0000:fffee000       .debug$S                   0000000180000000     dsound:DSOUND.dll
 0000:fffee000       .debug$S                   0000000180000000     dsound:DSOUND.dll
 0000:fffee000       .debug$S                   0000000180000000     dsound:DSOUND.dll
 0000:fffee000       .debug$S                   0000000180000000     dsound:DSOUND.dll
 0000:fffee000       .debug$S                   0000000180000000     kernel32:KERNEL32.dll
 0000:fffee000       .debug$S                   0000000180000000     kernel32:KERNEL32.dll
 0000:fffee000       .debug$S                   0000000180000000     kernel32:KERNEL32.dll
 0000:fffee000       .debug$S                   0000000180000000     kernel32:KERNEL32.dll
 0000:fffee000       .debug$S                   0000000180000000     kernel32:KERNEL32.dll
 0000:fffee000       .debug$S                   0000000180000000     kernel32:KERNEL32.dll
 0000:fffee000       .debug$S                   0000000180000000     kernel32:KERNEL32.dll
 0000:fffee000       .debug$S                   0000000180000000     kernel32:KERNEL32.dll
 0000:fffee000       .debug$S                   0000000180000000     kernel32:KERNEL32.dll
 0000:fffee000       .debug$S                   0000000180000000     kernel32:KERNEL32.dll
 0000:fffee000       .debug$S                   0000000180000000     kernel32:KERNEL32.dll
 0000:fffee000       .debug$S                   0000000180000000     kernel32:KERNEL32.dll
 0000:fffee000       .debug$S                   0000000180000000     kernel32:KERNEL32.dll
 0000:fffee000       .debug$S                   0000000180000000     kernel32:KERNEL32.dll
 0000:fffee000       .debug$S                   0000000180000000     kernel32:KERNEL32.dll
 0000:fffee000       .debug$S                   0000000180000000     kernel32:KERNEL32.dll
 0000:fffee000       .debug$S                   0000000180000000     kernel32:KERNEL32.dll
 0000:fffee000       .debug$S                   0000000180000000     kernel32:KERNEL32.dll
 0000:fffee000       .debug$S                   0000000180000000     kernel32:KERNEL32.dll
 0000:fffee000       .debug$S                   0000000180000000     kernel32:KERNEL32.dll
 0000:fffee000       .debug$S                   0000000180000000     kernel32:KERNEL32.dll
 0000:fffee000       .debug$S                   0000000180000000     kernel32:KERNEL32.dll
 0000:fffee000       .debug$S                   0000000180000000     kernel32:KERNEL32.dll
 0000:fffee000       .debug$S                   0000000180000000     kernel32:KERNEL32.dll
 0000:fffee000       .debug$S                   0000000180000000     kernel32:KERNEL32.dll
 0000:fffee000       .debug$S                   0000000180000000     kernel32:KERNEL32.dll
 0000:fffee000       .debug$S                   0000000180000000     kernel32:KERNEL32.dll
 0000:fffee000       .debug$S                   0000000180000000     kernel32:KERNEL32.dll
 0000:fffee000       .debug$S                   0000000180000000     ole32:ole32.dll
 0000:fffee000       .debug$S                   0000000180000000     ole32:ole32.dll
 0000:fffee000       .debug$S                   0000000180000000     user32:USER32.dll
 0000:fffee000       .debug$S                   0000000180000000     user32:USER32.dll
 0000:fffee000       .debug$S                   0000000180000000     winmm:WINMM.dll
 0000:fffee000       .debug$S                   0000000180000000     winmm:WINMM.dll
 0000:fffee000       .debug$S                   0000000180000000     winmm:WINMM.dll
 0000:fffee000       .debug$S                   0000000180000000     winmm:WINMM.dll
 0000:fffee000       .debug$S                   0000000180000000     winmm:WINMM.dll
 0000:fffee000       .debug$S                   0000000180000000     winmm:WINMM.dll
 0000:fffee000       .debug$S                   0000000180000000     winmm:WINMM.dll
 0000:fffee000       .debug$S                   0000000180000000     winmm:WINMM.dll
 0000:fffee000       .debug$S                   0000000180000000     winmm:WINMM.dll
 0000:fffee000       .debug$S                   0000000180000000     winmm:WINMM.dll
 0000:fffee000       .debug$S                   0000000180000000     winmm:WINMM.dll
 0000:fffee000       .debug$S                   0000000180000000     winmm:WINMM.dll
 0000:fffee000       .debug$S                   0000000180000000     winmm:WINMM.dll
 0000:fffee000       .debug$S                   0000000180000000     winmm:WINMM.dll
 0000:fffee000       .debug$S                   0000000180000000     winmm:WINMM.dll
 0000:fffee000       .debug$S                   0000000180000000     winmm:WINMM.dll
 0000:fffee000       .debug$S                   0000000180000000     winmm:WINMM.dll
 0000:fffee000       .debug$S                   0000000180000000     winmm:WINMM.dll
 0000:fffee000       .debug$S                   0000000180000000     winmm:WINMM.dll
 0000:fffee000       .debug$S                   0000000180000000     winmm:WINMM.dll
 0000:fffee000       .debug$S                   0000000180000000     winmm:WINMM.dll
 0000:fffee000       .debug$S                   0000000180000000     winmm:WINMM.dll
 0000:fffee000       .debug$S                   0000000180000000     winmm:WINMM.dll
 0000:fffee000       .debug$S                   0000000180000000     winmm:WINMM.dll
 0000:fffee000       .debug$S                   0000000180000000     winmm:WINMM.dll
 0000:fffee000       .debug$S                   0000000180000000     winmm:WINMM.dll
 0000:fffee000       .debug$S                   0000000180000000     winmm:WINMM.dll
 0000:fffee000       .debug$S                   0000000180000000     winmm:WINMM.dll
 0000:fffee000       .debug$S                   0000000180000000     winmm:WINMM.dll
 0000:fffee000       .debug$S                   0000000180000000     winmm:WINMM.dll
 0000:fffee000       .debug$S                   0000000180000000     winmm:WINMM.dll
 0000:fffee000       .debug$S                   0000000180000000     winmm:WINMM.dll
 0001:00000000       ??__E?data@DS_StartBufferHelper@@1VData@1@A@@YAXXZ 0000000180001000 f   PLATFORM_API_WinOS_DirectSound.obj
 0001:00000020       ??__E?data@MidiIn_OpenHelper@@1VData@1@A@@YAXXZ 0000000180001020 f   PLATFORM_API_WinOS_MidiIn.obj
 0001:00006c00       $$000000                   0000000180007c00     MSVCRT:amdsecgs.obj
 0001:00006fc0       ?dllmain_crt_dispatch@@YAHQEAUHINSTANCE__@@KQEAX@Z 0000000180007fc0 f   MSVCRT:dll_dllmain.obj
 0001:00007010       ?dllmain_crt_process_attach@@YAHQEAUHINSTANCE__@@QEAX@Z 0000000180008010 f   MSVCRT:dll_dllmain.obj
 0001:00007128       ?dllmain_crt_process_detach@@YAH_N@Z 0000000180008128 f   MSVCRT:dll_dllmain.obj
 0001:000071ac       ?dllmain_dispatch@@YAHQEAUHINSTANCE__@@KQEAX@Z 00000001800081ac f   MSVCRT:dll_dllmain.obj
 0001:00007428       capture_previous_context   0000000180008428 f   MSVCRT:gs_report.obj
 0001:00007be0       $$000000                   0000000180008be0     MSVCRT:guard_dispatch.obj
 0001:00007c00       $$000000                   0000000180008c00     MSVCRT:guard_xfg_dispatch.obj
 0001:00007c16       __scrt_is_nonwritable_in_current_image$filt$0 0000000180008c16 f   MSVCRT:utility.obj
 0001:00007c2e       ?fin$0@?0??dllmain_crt_process_attach@@YAHQEAUHINSTANCE__@@QEAX@Z@4HA 0000000180008c2e f   MSVCRT:dll_dllmain.obj
 0001:00007c45       ?fin$0@?0??dllmain_crt_process_detach@@YAH_N@Z@4HA 0000000180008c45 f   MSVCRT:dll_dllmain.obj
 0001:00007c5e       ?fin$1@?0??dllmain_crt_process_detach@@YAH_N@Z@4HA 0000000180008c5e f   MSVCRT:dll_dllmain.obj
 0001:00007c72       ?filt$0@?0??dllmain_dispatch@@YAHQEAUHINSTANCE__@@KQEAX@Z@4HA 0000000180008c72 f   MSVCRT:dll_dllmain.obj
 0001:00007ca8       ??__F?data@DS_StartBufferHelper@@1VData@1@A@@YAXXZ 0000000180008ca8 f   PLATFORM_API_WinOS_DirectSound.obj
 0001:00007cb4       ??__F?data@MidiIn_OpenHelper@@1VData@1@A@@YAXXZ 0000000180008cb4 f   PLATFORM_API_WinOS_MidiIn.obj
 0002:00000370       ??data$initializer$@DS_StartBufferHelper@@1P6AXXZEA@@3P6AXXZEA 0000000180009370     PLATFORM_API_WinOS_DirectSound.obj
 0002:00000378       ??data$initializer$@MidiIn_OpenHelper@@1P6AXXZEA@@3P6AXXZEA 0000000180009378     PLATFORM_API_WinOS_MidiIn.obj
 0002:00000938       GS_ExceptionPointers       0000000180009938     MSVCRT:gs_report.obj
 0002:00001260       $unwind$DAUDIO_AddAudioFormat 000000018000a260     DirectAudioDevice.obj
 0002:00001268       $unwind$Java_com_sun_media_sound_DirectAudioDevice_nGetFormats 000000018000a268     DirectAudioDevice.obj
 0002:00001274       $unwind$Java_com_sun_media_sound_DirectAudioDevice_nOpen 000000018000a274     DirectAudioDevice.obj
 0002:0000128c       $unwind$Java_com_sun_media_sound_DirectAudioDevice_nAvailable 000000018000a28c     DirectAudioDevice.obj
 0002:0000128c       $unwind$Java_com_sun_media_sound_DirectAudioDevice_nFlush 000000018000a28c     DirectAudioDevice.obj
 0002:0000128c       $unwind$Java_com_sun_media_sound_DirectAudioDevice_nGetBufferSize 000000018000a28c     DirectAudioDevice.obj
 0002:0000128c       $unwind$Java_com_sun_media_sound_DirectAudioDevice_nGetBytePosition 000000018000a28c     DirectAudioDevice.obj
 0002:0000128c       $unwind$Java_com_sun_media_sound_DirectAudioDevice_nRequiresServicing 000000018000a28c     DirectAudioDevice.obj
 0002:0000128c       $unwind$Java_com_sun_media_sound_DirectAudioDevice_nService 000000018000a28c     DirectAudioDevice.obj
 0002:0000128c       $unwind$Java_com_sun_media_sound_DirectAudioDevice_nSetBytePosition 000000018000a28c     DirectAudioDevice.obj
 0002:0000128c       $unwind$Java_com_sun_media_sound_DirectAudioDevice_nStart 000000018000a28c     DirectAudioDevice.obj
 0002:0000128c       $unwind$Java_com_sun_media_sound_DirectAudioDevice_nStop 000000018000a28c     DirectAudioDevice.obj
 0002:0000128c       $unwind$Java_com_sun_media_sound_MidiInDevice_nGetTimeStamp 000000018000a28c     MidiInDevice.obj
 0002:0000128c       $unwind$Java_com_sun_media_sound_MidiOutDevice_nGetTimeStamp 000000018000a28c     MidiOutDevice.obj
 0002:0000128c       $unwind$??__E?data@DS_StartBufferHelper@@1VData@1@A@@YAXXZ 000000018000a28c     PLATFORM_API_WinOS_DirectSound.obj
 0002:0000128c       $unwind$?ThreadProc@DS_StartBufferHelper@@KAKPEAX@Z 000000018000a28c     PLATFORM_API_WinOS_DirectSound.obj
 0002:0000128c       $unwind$DAUDIO_Stop        000000018000a28c     PLATFORM_API_WinOS_DirectSound.obj
 0002:0000128c       $unwind$??__E?data@MidiIn_OpenHelper@@1VData@1@A@@YAXXZ 000000018000a28c     PLATFORM_API_WinOS_MidiIn.obj
 0002:0000128c       $unwind$MIDI_IN_GetErrorStr 000000018000a28c     PLATFORM_API_WinOS_MidiIn.obj
 0002:0000128c       $unwind$MIDI_OUT_GetErrorStr 000000018000a28c     PLATFORM_API_WinOS_MidiOut.obj
 0002:0000128c       $unwind$MIDI_OUT_GetNumDevices 000000018000a28c     PLATFORM_API_WinOS_MidiOut.obj
 0002:0000128c       $unwind$getControlValue    000000018000a28c     PLATFORM_API_WinOS_Ports.obj
 0002:0000128c       $unwind$setControlValue    000000018000a28c     PLATFORM_API_WinOS_Ports.obj
 0002:0000128c       $unwind$MIDI_Lock          000000018000a28c     PLATFORM_API_WinOS_Util.obj
 0002:0000128c       $unwind$MIDI_Unlock        000000018000a28c     PLATFORM_API_WinOS_Util.obj
 0002:0000128c       $unwind$Java_com_sun_media_sound_PortMixer_nClose 000000018000a28c     PortMixer.obj
 0002:0000128c       $unwind$Java_com_sun_media_sound_PortMixer_nControlGetFloatValue 000000018000a28c     PortMixer.obj
 0002:0000128c       $unwind$Java_com_sun_media_sound_PortMixer_nControlGetIntValue 000000018000a28c     PortMixer.obj
 0002:0000128c       $unwind$Java_com_sun_media_sound_PortMixer_nControlSetFloatValue 000000018000a28c     PortMixer.obj
 0002:0000128c       $unwind$Java_com_sun_media_sound_PortMixer_nControlSetIntValue 000000018000a28c     PortMixer.obj
 0002:0000128c       $unwind$Java_com_sun_media_sound_PortMixer_nGetPortCount 000000018000a28c     PortMixer.obj
 0002:0000128c       $unwind$Java_com_sun_media_sound_PortMixer_nGetPortType 000000018000a28c     PortMixer.obj
 0002:0000128c       $unwind$__scrt_initialize_default_local_stdio_options 000000018000a28c     MSVCRT:default_local_stdio_options.obj
 0002:0000128c       $unwind$?dllmain_crt_dispatch@@YAHQEAUHINSTANCE__@@KQEAX@Z 000000018000a28c     MSVCRT:dll_dllmain.obj
 0002:0000128c       $unwind$DllMain            000000018000a28c     MSVCRT:dll_dllmain_stub.obj
 0002:0000128c       $unwind$__GSHandlerCheck   000000018000a28c     MSVCRT:gshandler.obj
 0002:0000128c       $unwind$__scrt_acquire_startup_lock 000000018000a28c     MSVCRT:utility.obj
 0002:0000128c       $unwind$__scrt_dllmain_after_initialize_c 000000018000a28c     MSVCRT:utility.obj
 0002:0000128c       $unwind$__scrt_dllmain_before_initialize_c 000000018000a28c     MSVCRT:utility.obj
 0002:0000128c       $unwind$__scrt_dllmain_crt_thread_attach 000000018000a28c     MSVCRT:utility.obj
 0002:0000128c       $unwind$__scrt_dllmain_crt_thread_detach 000000018000a28c     MSVCRT:utility.obj
 0002:0000128c       $unwind$__scrt_dllmain_uninitialize_c 000000018000a28c     MSVCRT:utility.obj
 0002:0000128c       $unwind$__scrt_dllmain_uninitialize_critical 000000018000a28c     MSVCRT:utility.obj
 0002:0000128c       $unwind$atexit             000000018000a28c     MSVCRT:utility.obj
 0002:00001294       $unwind$Java_com_sun_media_sound_DirectAudioDevice_nClose 000000018000a294     DirectAudioDevice.obj
 0002:00001294       $unwind$DAUDIO_Close       000000018000a294     PLATFORM_API_WinOS_DirectSound.obj
 0002:00001294       $unwind$MIDI_IN_ReleaseMessage 000000018000a294     PLATFORM_API_WinOS_MidiIn.obj
 0002:00001294       $unwind$MIDI_DestroyLock   000000018000a294     PLATFORM_API_WinOS_Util.obj
 0002:00001294       $unwind$MIDI_SetStartTime  000000018000a294     PLATFORM_API_WinOS_Util.obj
 0002:00001294       $unwind$MIDI_QueueClear    000000018000a294     PlatformMidi.obj
 0002:0000129c       $unwind$Java_com_sun_media_sound_DirectAudioDevice_nWrite 000000018000a29c     DirectAudioDevice.obj
 0002:000012c0       $unwind$Java_com_sun_media_sound_DirectAudioDevice_nRead 000000018000a2c0     DirectAudioDevice.obj
 0002:000012d8       $unwind$Java_com_sun_media_sound_DirectAudioDevice_nIsStillDraining 000000018000a2d8     DirectAudioDevice.obj
 0002:000012d8       $unwind$Java_com_sun_media_sound_MidiInDevice_nOpen 000000018000a2d8     MidiInDevice.obj
 0002:000012d8       $unwind$Java_com_sun_media_sound_MidiInDevice_nStart 000000018000a2d8     MidiInDevice.obj
 0002:000012d8       $unwind$Java_com_sun_media_sound_MidiOutDevice_nOpen 000000018000a2d8     MidiOutDevice.obj
 0002:000012d8       $unwind$??1Data@DS_StartBufferHelper@@QEAA@XZ 000000018000a2d8     PLATFORM_API_WinOS_DirectSound.obj
 0002:000012d8       $unwind$?DS_destroySoundBuffer@@YAXPEAUDS_Info@@@Z 000000018000a2d8     PLATFORM_API_WinOS_DirectSound.obj
 0002:000012d8       $unwind$?StartBuffer@DS_StartBufferHelper@@SAJPEAUDS_Info@@@Z 000000018000a2d8     PLATFORM_API_WinOS_DirectSound.obj
 0002:000012d8       $unwind$?isEqualGUID@@YAHPEAU_GUID@@0@Z 000000018000a2d8     PLATFORM_API_WinOS_DirectSound.obj
 0002:000012d8       $unwind$DAUDIO_Flush       000000018000a2d8     PLATFORM_API_WinOS_DirectSound.obj
 0002:000012d8       $unwind$??1Data@MidiIn_OpenHelper@@QEAA@XZ 000000018000a2d8     PLATFORM_API_WinOS_MidiIn.obj
 0002:000012d8       $unwind$?getMidiInCaps@@YAHHPEAUtagMIDIINCAPSW@@PEAH@Z 000000018000a2d8     PLATFORM_API_WinOS_MidiIn.obj
 0002:000012d8       $unwind$MIDI_IN_GetMessage 000000018000a2d8     PLATFORM_API_WinOS_MidiIn.obj
 0002:000012d8       $unwind$getMixerLineByDestination 000000018000a2d8     PLATFORM_API_WinOS_Ports.obj
 0002:000012d8       $unwind$getMixerLineBySource 000000018000a2d8     PLATFORM_API_WinOS_Ports.obj
 0002:000012d8       $unwind$MIDI_CreateLock    000000018000a2d8     PLATFORM_API_WinOS_Util.obj
 0002:000012d8       $unwind$MIDI_GetTimeStamp  000000018000a2d8     PLATFORM_API_WinOS_Util.obj
 0002:000012d8       $unwind$MIDI_WinDestroyLongBufferQueue 000000018000a2d8     PLATFORM_API_WinOS_Util.obj
 0002:000012d8       $unwind$MIDI_IN_InternalGetErrorString 000000018000a2d8     PlatformMidi.obj
 0002:000012d8       $unwind$MIDI_OUT_InternalGetErrorString 000000018000a2d8     PlatformMidi.obj
 0002:000012d8       $unwind$PORT_AddControl    000000018000a2d8     PortMixer.obj
 0002:000012d8       $unwind$__raise_securityfailure 000000018000a2d8     MSVCRT:gs_report.obj
 0002:000012d8       $unwind$??2@YAPEAX_K@Z     000000018000a2d8     MSVCRT:new_scalar.obj
 0002:000012d8       $unwind$??_Gtype_info@@UEAAPEAXI@Z 000000018000a2d8     MSVCRT:std_type_info_static.obj
 0002:000012d8       $unwind$??0bad_alloc@std@@QEAA@AEBV01@@Z 000000018000a2d8     MSVCRT:throw_bad_alloc.obj
 0002:000012d8       $unwind$??0bad_array_new_length@std@@QEAA@AEBV01@@Z 000000018000a2d8     MSVCRT:throw_bad_alloc.obj
 0002:000012d8       $unwind$??0exception@std@@QEAA@AEBV01@@Z 000000018000a2d8     MSVCRT:throw_bad_alloc.obj
 0002:000012d8       $unwind$__scrt_initialize_crt 000000018000a2d8     MSVCRT:utility.obj
 0002:000012d8       $unwind$__scrt_initialize_onexit_tables 000000018000a2d8     MSVCRT:utility.obj
 0002:000012d8       $unwind$__scrt_release_startup_lock 000000018000a2d8     MSVCRT:utility.obj
 0002:000012d8       $unwind$__scrt_uninitialize_crt 000000018000a2d8     MSVCRT:utility.obj
 0002:000012d8       $unwind$_onexit            000000018000a2d8     MSVCRT:utility.obj
 0002:000012e0       $unwind$handleGainAndConversion 000000018000a2e0     DirectAudioDevice.obj
 0002:000012f8       $unwind$Java_com_sun_media_sound_DirectAudioDeviceProvider_nNewDirectAudioDeviceInfo 000000018000a2f8     DirectAudioDeviceProvider.obj
 0002:0000131c       $unwind$getDirectAudioDeviceDescription 000000018000a31c     DirectAudioDeviceProvider.obj
 0002:0000131c       $unwind$?DS_GetDescEnum@@YAHPEAU_GUID@@PEBG1PEAUtag_DirectAudioDeviceDescription@@@Z 000000018000a31c     PLATFORM_API_WinOS_DirectSound.obj
 0002:0000131c       $unwind$?DS_RefreshCacheEnum@@YAHPEAU_GUID@@PEBD1PEAUDS_RefreshCacheStruct@@@Z 000000018000a31c     PLATFORM_API_WinOS_DirectSound.obj
 0002:0000131c       $unwind$?DS_removeDeviceRef@@YAXH@Z 000000018000a31c     PLATFORM_API_WinOS_DirectSound.obj
 0002:0000131c       $unwind$?midiInOpen@MidiIn_OpenHelper@@SAIHPEAUtag_MidiDeviceHandle@@@Z 000000018000a31c     PLATFORM_API_WinOS_MidiIn.obj
 0002:0000131c       $unwind$MIDI_IN_CloseDevice 000000018000a31c     PLATFORM_API_WinOS_MidiIn.obj
 0002:0000131c       $unwind$MIDI_IN_StartDevice 000000018000a31c     PLATFORM_API_WinOS_MidiIn.obj
 0002:0000131c       $unwind$getMidiOutCaps     000000018000a31c     PLATFORM_API_WinOS_MidiOut.obj
 0002:0000131c       $unwind$PORT_GetIntValue   000000018000a31c     PLATFORM_API_WinOS_Ports.obj
 0002:0000131c       $unwind$PORT_GetPortName   000000018000a31c     PLATFORM_API_WinOS_Ports.obj
 0002:0000131c       $unwind$MIDI_CreateQueue   000000018000a31c     PlatformMidi.obj
 0002:0000131c       $unwind$MIDI_QueueRead     000000018000a31c     PlatformMidi.obj
 0002:0000131c       $unwind$getPortMixerDescription 000000018000a31c     PortMixerProvider.obj
 0002:0000131c       $unwind$ThrowJavaMessageException 000000018000a31c     Utilities.obj
 0002:0000131c       $unwind$_RTC_Initialize    000000018000a31c     MSVCRT:initsect.obj
 0002:0000131c       $unwind$_RTC_Terminate     000000018000a31c     MSVCRT:initsect.obj
 0002:0000131c       $unwind$??_Gbad_alloc@std@@UEAAPEAXI@Z 000000018000a31c     MSVCRT:throw_bad_alloc.obj
 0002:0000131c       $unwind$??_Gbad_array_new_length@std@@UEAAPEAXI@Z 000000018000a31c     MSVCRT:throw_bad_alloc.obj
 0002:0000131c       $unwind$??_Gexception@std@@UEAAPEAXI@Z 000000018000a31c     MSVCRT:throw_bad_alloc.obj
 0002:00001328       $unwind$Java_com_sun_media_sound_MidiInDevice_nGetMessages 000000018000a328     MidiInDevice.obj
 0002:00001344       $unwind$Java_com_sun_media_sound_MidiInDeviceProvider_nGetDescription 000000018000a344     MidiInDeviceProvider.obj
 0002:00001344       $unwind$Java_com_sun_media_sound_MidiInDeviceProvider_nGetName 000000018000a344     MidiInDeviceProvider.obj
 0002:00001344       $unwind$Java_com_sun_media_sound_MidiInDeviceProvider_nGetVendor 000000018000a344     MidiInDeviceProvider.obj
 0002:00001344       $unwind$Java_com_sun_media_sound_MidiInDeviceProvider_nGetVersion 000000018000a344     MidiInDeviceProvider.obj
 0002:00001344       $unwind$Java_com_sun_media_sound_MidiOutDeviceProvider_nGetDescription 000000018000a344     MidiOutDeviceProvider.obj
 0002:00001344       $unwind$Java_com_sun_media_sound_MidiOutDeviceProvider_nGetName 000000018000a344     MidiOutDeviceProvider.obj
 0002:00001344       $unwind$Java_com_sun_media_sound_MidiOutDeviceProvider_nGetVendor 000000018000a344     MidiOutDeviceProvider.obj
 0002:00001344       $unwind$Java_com_sun_media_sound_MidiOutDeviceProvider_nGetVersion 000000018000a344     MidiOutDeviceProvider.obj
 0002:00001358       $unwind$Java_com_sun_media_sound_MidiOutDevice_nSendLongMessage 000000018000a358     MidiOutDevice.obj
 0002:00001358       $unwind$?findCacheItemByGUID@@YAHPEAU_GUID@@H@Z 000000018000a358     PLATFORM_API_WinOS_DirectSound.obj
 0002:00001358       $unwind$unprepareLongBuffers 000000018000a358     PLATFORM_API_WinOS_MidiOut.obj
 0002:00001358       $unwind$addAllControls     000000018000a358     PLATFORM_API_WinOS_Ports.obj
 0002:00001358       $unwind$MIDI_QueueAddLong  000000018000a358     PlatformMidi.obj
 0002:00001358       $unwind$MIDI_QueueAddShort 000000018000a358     PlatformMidi.obj
 0002:00001358       $unwind$__scrt_dllmain_exception_filter 000000018000a358     MSVCRT:utility.obj
 0002:0000136c       $unwind$UnicodeToUTF8      000000018000a36c     PLATFORM_API_WinOS_Charset_Util.obj
 0002:00001380       $unwind$UnicodeToUTF8AndCopy 000000018000a380     PLATFORM_API_WinOS_Charset_Util.obj
 0002:00001380       $unwind$DAUDIO_GetDirectAudioDeviceDescription 000000018000a380     PLATFORM_API_WinOS_DirectSound.obj
 0002:00001380       $unwind$?unprepareBuffers@@YAHPEAUtag_MidiDeviceHandle@@@Z 000000018000a380     PLATFORM_API_WinOS_MidiIn.obj
 0002:00001380       $unwind$MIDI_IN_StopDevice 000000018000a380     PLATFORM_API_WinOS_MidiIn.obj
 0002:00001380       $unwind$MIDI_OUT_CloseDevice 000000018000a380     PLATFORM_API_WinOS_MidiOut.obj
 0002:00001380       $unwind$freeLongBuffer     000000018000a380     PLATFORM_API_WinOS_MidiOut.obj
 0002:00001380       $unwind$freeLongBuffers    000000018000a380     PLATFORM_API_WinOS_MidiOut.obj
 0002:00001380       $unwind$PORT_SetIntValue   000000018000a380     PLATFORM_API_WinOS_Ports.obj
 0002:00001380       $unwind$_DllMainCRTStartup 000000018000a380     MSVCRT:dll_dllmain.obj
 0002:00001390       $unwind$DAUDIO_GetDirectAudioDeviceCount 000000018000a390     PLATFORM_API_WinOS_DirectSound.obj
 0002:0000139c       $unwind$DAUDIO_GetFormats  000000018000a39c     PLATFORM_API_WinOS_DirectSound.obj
 0002:000013b8       $unwind$DAUDIO_Open        000000018000a3b8     PLATFORM_API_WinOS_DirectSound.obj
 0002:000013b8       $unwind$PORT_NewBooleanControl 000000018000a3b8     PortMixer.obj
 0002:000013cc       $unwind$DAUDIO_Start       000000018000a3cc     PLATFORM_API_WinOS_DirectSound.obj
 0002:000013d8       $unwind$DAUDIO_Write       000000018000a3d8     PLATFORM_API_WinOS_DirectSound.obj
 0002:000013f0       $unwind$DAUDIO_Read        000000018000a3f0     PLATFORM_API_WinOS_DirectSound.obj
 0002:00001404       $unwind$??0Data@DS_StartBufferHelper@@QEAA@XZ 000000018000a404     PLATFORM_API_WinOS_DirectSound.obj
 0002:00001404       $unwind$DAUDIO_StillDraining 000000018000a404     PLATFORM_API_WinOS_DirectSound.obj
 0002:00001404       $unwind$??0Data@MidiIn_OpenHelper@@QEAA@XZ 000000018000a404     PLATFORM_API_WinOS_MidiIn.obj
 0002:00001404       $unwind$?MIDI_IN_PutMessage@@YAXPEAUHMIDIIN__@@I_K11@Z 000000018000a404     PLATFORM_API_WinOS_MidiIn.obj
 0002:0000140c       $unwind$DAUDIO_GetAvailable 000000018000a40c     PLATFORM_API_WinOS_DirectSound.obj
 0002:00001414       $unwind$DAUDIO_GetBytePosition 000000018000a414     PLATFORM_API_WinOS_DirectSound.obj
 0002:00001420       $unwind$DAUDIO_Service     000000018000a420     PLATFORM_API_WinOS_DirectSound.obj
 0002:00001428       $unwind$?DS_addDeviceRef@@YAHH@Z 000000018000a428     PLATFORM_API_WinOS_DirectSound.obj
 0002:00001438       $unwind$?DS_clearBuffer@@YAXPEAUDS_Info@@H@Z 000000018000a438     PLATFORM_API_WinOS_DirectSound.obj
 0002:00001448       $unwind$?DS_createSoundBuffer@@YAPEAXPEAUDS_Info@@MHHH@Z 000000018000a448     PLATFORM_API_WinOS_DirectSound.obj
 0002:00001468       $unwind$?DS_GetAvailable@@YAHPEAUDS_Info@@PEAK1PEAHH@Z 000000018000a468     PLATFORM_API_WinOS_DirectSound.obj
 0002:0000147c       $unwind$snprintf           000000018000a47c     PLATFORM_API_WinOS_MidiIn.obj
 0002:0000148c       $unwind$MIDI_IN_GetDeviceName 000000018000a48c     PLATFORM_API_WinOS_MidiIn.obj
 0002:000014a4       $unwind$MIDI_IN_GetDeviceVersion 000000018000a4a4     PLATFORM_API_WinOS_MidiIn.obj
 0002:000014a4       $unwind$MIDI_OUT_GetDeviceDescription 000000018000a4a4     PLATFORM_API_WinOS_MidiOut.obj
 0002:000014a4       $unwind$MIDI_OUT_GetDeviceName 000000018000a4a4     PLATFORM_API_WinOS_MidiOut.obj
 0002:000014bc       $unwind$MIDI_IN_OpenDevice 000000018000a4bc     PLATFORM_API_WinOS_MidiIn.obj
 0002:000014d4       $unwind$?ThreadProc@MidiIn_OpenHelper@@KAKPEAX@Z 000000018000a4d4     PLATFORM_API_WinOS_MidiIn.obj
 0002:000014dc       $unwind$MIDI_OUT_GetDeviceVersion 000000018000a4dc     PLATFORM_API_WinOS_MidiOut.obj
 0002:000014f4       $unwind$MIDI_OUT_OpenDevice 000000018000a4f4     PLATFORM_API_WinOS_MidiOut.obj
 0002:00001500       $unwind$MIDI_OUT_SendLongMessage 000000018000a500     PLATFORM_API_WinOS_MidiOut.obj
 0002:0000151c       $unwind$PORT_GetPortMixerDescription 000000018000a51c     PLATFORM_API_WinOS_Ports.obj
 0002:00001530       $unwind$PORT_Open          000000018000a530     PLATFORM_API_WinOS_Ports.obj
 0002:00001548       $unwind$PORT_Close         000000018000a548     PLATFORM_API_WinOS_Ports.obj
 0002:00001550       $unwind$PORT_GetControls   000000018000a550     PLATFORM_API_WinOS_Ports.obj
 0002:0000156c       $unwind$PORT_GetFloatValue 000000018000a56c     PLATFORM_API_WinOS_Ports.obj
 0002:0000157c       $unwind$PORT_SetFloatValue 000000018000a57c     PLATFORM_API_WinOS_Ports.obj
 0002:00001588       $unwind$getControlInfo     000000018000a588     PLATFORM_API_WinOS_Ports.obj
 0002:00001598       $unwind$lineHasControls    000000018000a598     PLATFORM_API_WinOS_Ports.obj
 0002:000015a4       $unwind$getDestinationCount 000000018000a5a4     PLATFORM_API_WinOS_Ports.obj
 0002:000015b4       $unwind$getControlCount    000000018000a5b4     PLATFORM_API_WinOS_Ports.obj
 0002:000015c4       $unwind$createMuxControl   000000018000a5c4     PLATFORM_API_WinOS_Ports.obj
 0002:000015e0       $unwind$createPortControl  000000018000a5e0     PLATFORM_API_WinOS_Ports.obj
 0002:000015ec       $unwind$createLineControls 000000018000a5ec     PLATFORM_API_WinOS_Ports.obj
 0002:00001608       $unwind$MIDI_WinCreateLongBufferQueue 000000018000a608     PLATFORM_API_WinOS_Util.obj
 0002:00001624       $unwind$MIDI_DestroyQueue  000000018000a624     PlatformMidi.obj
 0002:00001624       $unwind$MIDI_QueueRemove   000000018000a624     PlatformMidi.obj
 0002:00001630       $unwind$Java_com_sun_media_sound_PortMixer_nGetPortName 000000018000a630     PortMixer.obj
 0002:00001644       $unwind$Java_com_sun_media_sound_PortMixer_nGetControls 000000018000a644     PortMixer.obj
 0002:0000165c       $unwind$PORT_NewCompoundControl 000000018000a65c     PortMixer.obj
 0002:00001678       $unwind$PORT_NewFloatControl 000000018000a678     PortMixer.obj
 0002:00001694       $unwind$Java_com_sun_media_sound_PortMixerProvider_nNewPortMixerInfo 000000018000a694     PortMixerProvider.obj
 0002:000016b8       $unwind$__GSHandlerCheckCommon 000000018000a6b8     MSVCRT:gshandler.obj
 0002:000016c0       $xdatasym                  000000018000a6c0     MSVCRT:amdsecgs.obj
 0002:000016c4       $unwind$__scrt_is_nonwritable_in_current_image 000000018000a6c4     MSVCRT:utility.obj
 0002:000016e4       $unwind$__scrt_is_nonwritable_in_current_image$filt$0 000000018000a6e4     MSVCRT:utility.obj
 0002:000016ec       $unwind$?dllmain_crt_process_attach@@YAHQEAUHINSTANCE__@@QEAX@Z 000000018000a6ec     MSVCRT:dll_dllmain.obj
 0002:00001728       $unwind$?fin$0@?0??dllmain_crt_process_attach@@YAHQEAUHINSTANCE__@@QEAX@Z@4HA 000000018000a728     MSVCRT:dll_dllmain.obj
 0002:00001728       $unwind$?fin$0@?0??dllmain_crt_process_detach@@YAH_N@Z@4HA 000000018000a728     MSVCRT:dll_dllmain.obj
 0002:00001728       $unwind$?fin$1@?0??dllmain_crt_process_detach@@YAH_N@Z@4HA 000000018000a728     MSVCRT:dll_dllmain.obj
 0002:00001730       $unwind$?dllmain_crt_process_detach@@YAH_N@Z 000000018000a730     MSVCRT:dll_dllmain.obj
 0002:00001784       $unwind$?dllmain_dispatch@@YAHQEAUHINSTANCE__@@KQEAX@Z 000000018000a784     MSVCRT:dll_dllmain.obj
 0002:000017ac       $unwind$?filt$0@?0??dllmain_dispatch@@YAHQEAUHINSTANCE__@@KQEAX@Z@4HA 000000018000a7ac     MSVCRT:dll_dllmain.obj
 0002:000017b4       $unwind$__report_gsfailure 000000018000a7b4     MSVCRT:gs_report.obj
 0002:000017bc       $unwind$capture_previous_context 000000018000a7bc     MSVCRT:gs_report.obj
 0002:000017c8       $unwind$__isa_available_init 000000018000a7c8     MSVCRT:cpu_disp.obj
 0002:000017d8       $unwind$__scrt_fastfail    000000018000a7d8     MSVCRT:utility_desktop.obj
 0002:000017e8       $unwind$__security_init_cookie 000000018000a7e8     MSVCRT:gs_support.obj
 0002:000017f4       $unwind$?__scrt_throw_std_bad_alloc@@YAXXZ 000000018000a7f4     MSVCRT:throw_bad_alloc.obj
 0002:000017f4       $unwind$?__scrt_throw_std_bad_array_new_length@@YAXXZ 000000018000a7f4     MSVCRT:throw_bad_alloc.obj
 0002:00001800       $xdatasym                  000000018000a800     MSVCRT:guard_dispatch.obj
 0002:00001808       $xdatasym                  000000018000a808     MSVCRT:guard_xfg_dispatch.obj
 0002:00001900       .edata                     000000018000a900     jsound.exp
 0002:00001928       rgpv                       000000018000a928     jsound.exp
 0002:000019f4       rgszName                   000000018000a9f4     jsound.exp
 0002:00001ac0       rgwOrd                     000000018000aac0     jsound.exp
 0002:00001b26       szName                     000000018000ab26     jsound.exp
 0002:00001b31       $N00001                    000000018000ab31     jsound.exp
 0002:00001b73       $N00002                    000000018000ab73     jsound.exp
 0002:00001bc0       $N00003                    000000018000abc0     jsound.exp
 0002:00001bf6       $N00004                    000000018000abf6     jsound.exp
 0002:00001c28       $N00005                    000000018000ac28     jsound.exp
 0002:00001c5a       $N00006                    000000018000ac5a     jsound.exp
 0002:00001c94       $N00007                    000000018000ac94     jsound.exp
 0002:00001cd0       $N00008                    000000018000acd0     jsound.exp
 0002:00001d07       $N00009                    000000018000ad07     jsound.exp
 0002:00001d43       $N00010                    000000018000ad43     jsound.exp
 0002:00001d74       $N00011                    000000018000ad74     jsound.exp
 0002:00001da5       $N00012                    000000018000ada5     jsound.exp
 0002:00001de3       $N00013                    000000018000ade3     jsound.exp
 0002:00001e17       $N00014                    000000018000ae17     jsound.exp
 0002:00001e53       $N00015                    000000018000ae53     jsound.exp
 0002:00001e85       $N00016                    000000018000ae85     jsound.exp
 0002:00001eb6       $N00017                    000000018000aeb6     jsound.exp
 0002:00001ee8       $N00018                    000000018000aee8     jsound.exp
 0002:00001f26       $N00019                    000000018000af26     jsound.exp
 0002:00001f5d       $N00020                    000000018000af5d     jsound.exp
 0002:00001f9a       $N00021                    000000018000af9a     jsound.exp
 0002:00001fd3       $N00022                    000000018000afd3     jsound.exp
 0002:0000200d       $N00023                    000000018000b00d     jsound.exp
 0002:0000203a       $N00024                    000000018000b03a     jsound.exp
 0002:0000206d       $N00025                    000000018000b06d     jsound.exp
 0002:000020a1       $N00026                    000000018000b0a1     jsound.exp
 0002:000020cd       $N00027                    000000018000b0cd     jsound.exp
 0002:000020fa       $N00028                    000000018000b0fa     jsound.exp
 0002:00002126       $N00029                    000000018000b126     jsound.exp
 0002:00002165       $N00030                    000000018000b165     jsound.exp
 0002:0000219d       $N00031                    000000018000b19d     jsound.exp
 0002:000021db       $N00032                    000000018000b1db     jsound.exp
 0002:00002215       $N00033                    000000018000b215     jsound.exp
 0002:00002250       $N00034                    000000018000b250     jsound.exp
 0002:0000227e       $N00035                    000000018000b27e     jsound.exp
 0002:000022b3       $N00036                    000000018000b2b3     jsound.exp
 0002:000022e0       $N00037                    000000018000b2e0     jsound.exp
 0002:00002318       $N00038                    000000018000b318     jsound.exp
 0002:00002351       $N00039                    000000018000b351     jsound.exp
 0002:00002380       $N00040                    000000018000b380     jsound.exp
 0002:000023ba       $N00041                    000000018000b3ba     jsound.exp
 0002:000023f7       $N00042                    000000018000b3f7     jsound.exp
 0002:00002421       $N00043                    000000018000b421     jsound.exp
 0002:0000245a       $N00044                    000000018000b45a     jsound.exp
 0002:00002491       $N00045                    000000018000b491     jsound.exp
 0002:000024ca       $N00046                    000000018000b4ca     jsound.exp
 0002:00002501       $N00047                    000000018000b501     jsound.exp
 0002:00002531       $N00048                    000000018000b531     jsound.exp
 0002:00002562       $N00049                    000000018000b562     jsound.exp
 0002:00002592       $N00050                    000000018000b592     jsound.exp
 0002:000025c2       $N00051                    000000018000b5c2     jsound.exp
 0002:000029f8       .idata$6                   000000018000b9f8     dsound:DSOUND.dll
 0002:00002c5e       .idata$6                   000000018000bc5e     winmm:WINMM.dll
 0002:00002c92       .idata$6                   000000018000bc92     user32:USER32.dll
 0002:00002cc0       .idata$6                   000000018000bcc0     ole32:ole32.dll
 0002:00002f02       .idata$6                   000000018000bf02     kernel32:KERNEL32.dll
 0002:00002fae       .idata$6                   000000018000bfae     vcruntime:VCRUNTIME140.dll
 0002:000030dc       .idata$6                   000000018000c0dc     ucrt:api-ms-win-crt-heap-l1-1-0.dll
 0002:000030fc       .idata$6                   000000018000c0fc     ucrt:api-ms-win-crt-string-l1-1-0.dll
 0002:0000311e       .idata$6                   000000018000c11e     ucrt:api-ms-win-crt-stdio-l1-1-0.dll
 0002:0000313e       .idata$6                   000000018000c13e     ucrt:api-ms-win-crt-runtime-l1-1-0.dll
 0003:00000000       ?sampleRateArray@@3PAHA    000000018000d000     PLATFORM_API_WinOS_DirectSound.obj
 0003:00000008       ?channelsArray@@3PAHA      000000018000d008     PLATFORM_API_WinOS_DirectSound.obj
 0003:00000010       ?bitsArray@@3PAHA          000000018000d010     PLATFORM_API_WinOS_DirectSound.obj
 0003:00000150       ?g_audioDeviceCache@@3PAUDS_AudioDeviceCache@@A 000000018000d150     PLATFORM_API_WinOS_DirectSound.obj
 0003:00000ab0       ?g_cacheCount@@3HA         000000018000dab0     PLATFORM_API_WinOS_DirectSound.obj
 0003:00000ab4       ?g_mixerCount@@3HA         000000018000dab4     PLATFORM_API_WinOS_DirectSound.obj
 0003:00000ab8       ?g_lastCacheRefreshTime@@3_KA 000000018000dab8     PLATFORM_API_WinOS_DirectSound.obj
 0003:00000ac0       ?CLSID_DAUDIO_Zero@@3U_GUID@@A 000000018000dac0     PLATFORM_API_WinOS_DirectSound.obj
 0003:00000b30       ?winMidiInErrMsg@@3PADA    000000018000db30     PLATFORM_API_WinOS_MidiIn.obj
 0003:00000c00       winMidiOutErrMsg           000000018000dc00     PLATFORM_API_WinOS_MidiOut.obj
 0003:00000cd8       ?is_initialized_as_dll@@3_NA 000000018000dcd8     MSVCRT:utility.obj
 0003:00000cd9       ?module_local_atexit_table_initialized@@3_NA 000000018000dcd9     MSVCRT:utility.obj
 0003:00000ce0       ?module_local_atexit_table@@3U_onexit_table_t@@A 000000018000dce0     MSVCRT:utility.obj
 0003:00000cf8       ?module_local_at_quick_exit_table@@3U_onexit_table_t@@A 000000018000dcf8     MSVCRT:utility.obj
 0003:00000d10       ?__proc_attached@@3HA      000000018000dd10     MSVCRT:dll_dllmain.obj
 0003:00000d20       GS_ExceptionRecord         000000018000dd20     MSVCRT:gs_report.obj
 0003:00000dc0       GS_ContextRecord           000000018000ddc0     MSVCRT:gs_report.obj
 0005:00000060       $R000000                   0000000180010060     jsound.dll.res
